:100000000C94FF030C941E040C941E040C941E0408
:100010000C941E040C941E040C941E040C941E04D8
:100020000C941E040C941E040C9494120C941E0444
:100030000C941E040C941E040C941E040C941E04B8
:100040000C942D1D0C941E040C941E040C941E0480
:100050000C94D31D0C9435150C941E040C941E04A2
:100060000C941E040C941E040C941E040C941E0488
:100070000C941E040C941E040C941E040C941E0478
:100080000C941E040C941E040C941E040C941E0468
:100090000C941E040C941E0453797374656D206FC8
:1000A0006E6C696E652E0A000A0A0A2A2A2A2A2A12
:1000B0002A2A2A424F4F54494E4720434F4E544913
:1000C0004B492A2A2A2A2A2A2A2A2A0A0025632070
:1000D0006973206E6F7420612076616C6964206F93
:1000E0007074696F6E21206820666F72206D656E76
:1000F000750A0D0020202A204F70657261746573A7
:10010000206F6E206368616E6E656C2025640A0D39
:10011000004F757470757420726177203830322EFC
:1001200031352E34206672616D65730A0D20006EC4
:100130006F7420006465636F6D7072657373203631
:100140006C6F7770616E20686561646572730A0D0B
:1001500020202A2057696C6C20006E6F7420006389
:1001600068616E6765206C696E6B2D6C6F63616C86
:100170002061646472657373657320696E7369646A
:1001800065204950206D657373616765730A0D20A2
:10019000202A2057696C6C20006E6F7420007365F4
:1001A0006E642064617461206F7665722052460A25
:1001B0000D20202A2057696C6C20006E6F7420007F
:1001C00043757272656E746C79204A61636B646109
:1001D000773A0A0D20202A2057696C6C200053655D
:1001E0006C656374203830322E31352E34204368EC
:1001F000616E6E656C20696E2072616E676520317C
:10020000312D3236205B25645D3A20004A61636BF4
:10021000646177206E6F77206361707475726573A7
:1002200020726177206672616D65730A0D004A6104
:10023000636B64617720646F6573206E6F742063F5
:1002400061707475726520726177206672616D6588
:10025000730A0D004A61636B646177206E6F7720CB
:10026000706572666F726D7320366C6F7770616E39
:10027000207472616E736C6174696F6E730A0D0025
:100280004A61636B64617720646F6573206E6F747D
:1002900020706572666F726D20366C6F7770616E5C
:1002A000207472616E736C6174696F6E0A0D004A1E
:1002B00061636B646177206E6F7720696E206E6575
:1002C00074776F726B206D6F64650A0D004A61630D
:1002D0006B646177206E6F7720696E20736E69663C
:1002E000666572206D6F64650A0D000A0D496E70B7
:1002F000757420746F6F206C6F6E67210A0D000A91
:100300000D496E76616C696420696E7075740A0DB2
:10031000002A2A2A2A2A2A2A2A2A2A2A2A2A2A2A67
:100320002A2A2A2A2A2A2A2A2A2A2A2A2A2A2A2A2D
:100330002A2A2A2A2A2A2A2A2A2A2A0A0D002A208E
:10034000796F75722063686F696365206F6E206BCB
:100350006579626F6172642E202020202020202089
:10036000202020202020202A0A0D002A204D616B09
:10037000652073656C656374696F6E2061742061BC
:100380006E792074696D652062792070726573736F
:10039000696E67202A0A0D002A20202020202020B4
:1003A000202020202020202020202020202020204D
:1003B000202020202020202020202020202020203D
:1003C000202A0A0D002A202075202020202020200D
:1003D0002020202020202020537769746368207417
:1003E0006F206D6173732D73746F726167652A0A74
:1003F0000D002A20207220202020202020202020D4
:100400002020202020546F67676C65207261772060
:100410006D6F6465202020202020202A0A0D002AEC
:1004200020203620202020202020202020202020B6
:100430002020546F67676C6520366C6F7770616E33
:1004400020202020202020202A0A0D002A2020639E
:100450002020202020202020202020202020205369
:100460006574205246206368616E6E656C202020A2
:1004700020202020202A0A0D002A20206E20202063
:1004800020202020202020202020202053657420A0
:10049000746F206E6574776F726B206D6F6465206A
:1004A00020202A0A0D002A2020732020202020202E
:1004B00020202020202020202053657420746F20CD
:1004C000736E6966666572206D6F64652020202AF0
:1004D0000A0D002A20206D2020202020202020200E
:1004E0002020202020205072696E74206375727263
:1004F000656E74206D6F6465202020202A0A0D002F
:100500002A2020682C3F202020202020202020206E
:100510002020205072696E742074686973206D65A4
:100520006E75202020202020202A0A0D002A204D30
:1005300061696E204D656E753A20202020202020B4
:1005400020202020202020202020202020202020AB
:100550002020202020202A0A0D002A2020202020D0
:10056000202020202020202020202020202020208B
:10057000202020202020202020202020202020207B
:100580002020202A0A0D000A0A0D2A2A2A2A2A2AAD
:100590002A2A2A2A204A61636B646177204D656E9E
:1005A00075202A2A2A2A2A2A2A2A2A2A2A2A2A2A6A
:1005B0002A2A2A2A0A0D0001010100020101000372
:1005C0000101000401010006010100070101000A08
:1005D0000101000B0101000C0101000D0101000EE1
:1005E00001010011010100140101001601010002C6
:1005F00002010001010200020102000301020004E5
:10060000010200050102001B0201000101010102BB
:1006100001010103010101040101010501010101C1
:100620000102010201020103010201000101FD02B8
:100630000101FD010101FD060101FD030101FD04B0
:100640000101FD7261776D6F64650050414E494450
:100650003A203078424141440041746D656C00009D
:1006600000000012010002EF020140EB0321200014
:10067000100102030109028D000401008032080B01
:1006800000020202FF0009040000010202FF00054F
:1006900024001001052401000104240200052406A1
:1006A00000010705810308000109040100020A0096
:1006B0000000070582024000000705030240000019
:1006C000080B0202020201000904020001020201F9
:1006D0000005240010010524010303042402000581
:1006E00024060203070584032000FF090403000217
:1006F0000A00000007058502200000070506022009
:100700000000120100020202FF40EB03192000105A
:1007100001020301090243000201008032090400C2
:1007200000010202FF000524001001052401000160
:1007300004240200052406000107058103080001C6
:1007400009040100020A00000007058202400000BF
:10075000070503024000001201000200000040EB08
:10076000032F2000100102030109022000010100F3
:10077000803209040000020806500007058102408B
:100780000000070502024000000C03410074006DE8
:100790000065006C00220352005A005200410056CE
:1007A0000045004E00200055005300420020004448
:1007B0000045004D004F000C0331002E0030002E8C
:1007C0000030000403090441544D454C20202052C0
:1007D0005A524156454E55534220444F43532030C0
:1007E0002E3030008000021F0000002241565220AF
:1007F000466C617368204D656D6F7279220011241B
:100800001FBECFEFD0E2DEBFCDBF13E0A0E0B1E06E
:10081000EEE3F6E900E00BBF02C007900D92A031B5
:10082000B107D9F713E1A0E1B3E001C01D92A43AEA
:10083000B107E1F70E9420040C941D4B0C940000BA
:1008400011240E9416310E94CB1400D088EA90E057
:10085000EDB7FEB7928381830E948B470F900F9074
:100860000E94DE230E940D2584E591E060E070E0A7
:100870000E94CA2489E191E060E070E00E94CA24ED
:1008800081E391E060E070E00E94CA248EE691E08E
:1008900060E070E00E94CA2400D088E990E0EDB7E3
:1008A000FEB7928381830E948B470F900F900E9426
:1008B00029310E94EE23FDCF76988AE08093760B53
:1008C000089500D087E895E0EDB7FEB79283818365
:1008D0000E948B478AE595E0EDB7FEB7928381834E
:1008E0000E948B478DE295E0EDB7FEB7928381833E
:1008F0000E948B4780E095E0EDB7FEB7928381833D
:100900000E948B4783ED94E0EDB7FEB7928381831D
:100910000E948B4786EA94E0EDB7FEB7928381830D
:100920000E948B4789E794E0EDB7FEB792838183FD
:100930000E948B478CE494E0EDB7FEB792838183ED
:100940000E948B478FE194E0EDB7FEB792838183DD
:100950000E948B4782EF93E0EDB7FEB792838183CD
:100960000E948B4785EC93E0EDB7FEB792838183BD
:100970000E948B4788E993E0EDB7FEB792838183AD
:100980000E948B478BE693E0EDB7FEB7928381839D
:100990000E948B478EE393E0EDB7FEB7928381838D
:1009A0000E948B4781E193E0EDB7FEB7928381838C
:1009B0000E948B470F900F9008951F93CF93DF9362
:1009C000282F8091150390911603019709F072C0AA
:1009D0002A3041F02D3031F080911103283009F098
:1009E0004EC048C010911103E12FF0E0EE5EFC4FC5
:1009F000108282E193E00E94FB46EC01112319F082
:100A00008B3091051CF0CB31D1056CF000D08FEF0D
:100A100092E0ADB7BEB712969C938E9311970E9449
:100A20008B470F900F90209701F11C2F8C2F0E9465
:100A30004B19F999FECF1FBA89E090E092BD81BDB4
:100A400010BD0FB6F894FA9AF99A0FBEF999FECF35
:100A50001FBA8AE090E092BD81BDFE01E095E0BD45
:100A60000FB6F894FA9AF99A0FBE109216031092E4
:100A7000150395C1882309F492C1815018C08230B2
:100A800080F0109216031092150300D08BEE92E0C6
:100A9000ADB7BEB712969C938E9311970E948B4769
:100AA00091C0E82FF0E0EE5EFC4F20838F5F8093D3
:100AB000110375C1283631F1293694F4263309F42F
:100AC00040C027333CF42A3009F469C12D3009F0C5
:100AD00052C165C12F33B1F0233609F04CC175C046
:100AE000223709F44EC023373CF42D3609F489C06F
:100AF0002E3609F040C116C0233739F0253709F0EA
:100B00003AC10CC10E9461044AC100D08DEC92E050
:100B1000EDB7FEB7928381830E948B478091D612F6
:100B2000897F4EC000D08FEA92E0ADB7BEB7129673
:100B30009C938E9311970E948B478091D61286606A
:100B40003FC08091D61280FF0DC000D080E892E0B7
:100B5000EDB7FEB7928381830E948B478091D612B6
:100B60008E7F2EC000D084E592E0ADB7BEB712965E
:100B70009C938E9311970E948B478091D61281602F
:100B80001FC08091D61283FF0DC000D08EE292E08C
:100B9000EDB7FEB7928381830E948B478091D61276
:100BA000877F0EC000D08CE092E0ADB7BEB7129642
:100BB0009C938E9311970E948B478091D6128860E8
:100BC0008093D6120F900F90EAC00E94451900D072
:100BD00000D0EDB7FEB731962EED31E0ADB7BEB720
:100BE00012963C932E931197828313820E948B4717
:100BF00081E090E090931603809315031092110307
:100C0000CAC000D080EC91E0EDB7FEB7928381833B
:100C10000E948B478091D6120F900F9081FD0DC0DE
:100C200000D08BEB91E0ADB7BEB712969C938E933C
:100C300011970E948B470F900F9000D08EE991E0A2
:100C4000EDB7FEB7928381830E948B478091D612C5
:100C50000F900F9082FD0DC000D089E991E0ADB7F3
:100C6000BEB712969C938E9311970E948B470F905C
:100C70000F9000D08FE591E0EDB7FEB792838183AE
:100C80000E948B478091D6120F900F9080FD0DC06F
:100C900000D08AE591E0ADB7BEB712969C938E93D3
:100CA00011970E948B470F900F9000D084E391E042
:100CB000EDB7FEB7928381830E948B478091D61255
:100CC0000F900F9083FD0DC000D08FE291E0ADB783
:100CD000BEB712969C938E9311970E948B470F90EC
:100CE0000F9000D081E191E0EDB7FEB79283818350
:100CF0000E948B470F900F900E94451900D000D0A2
:100D0000EDB7FEB7319624EF30E0ADB7BEB712961F
:100D10003C932E931197828313823BC082E090E034
:100D200090934701809346011092A1131092A01353
:100D30001092660C1092650C5F985D9A8EB1806C73
:100D40008EB98091E00081608093E00020E048EC63
:100D500050E008C0FA013197F1F70197D9F72F5FFA
:100D6000223319F088EE93E0F5CF8091E0008E7F7A
:100D70008093E00014C000D000D08DEC90E0EDB77F
:100D8000FEB792838183822F992787FD9095948364
:100D900083830E948B470F900F900F900F90DF91ED
:100DA000CF911F910895CF93DF93EC0188819981B2
:100DB000009729F0813A910509F062C058C00E945D
:100DC0001B368091760B882321F081508093760B1F
:100DD00001C0769A8091790C882399F1809146011F
:100DE00090914701019769F58091650C9091660C8F
:100DF000892B39F180911F03882319F580910C010B
:100E0000882331F00E9420360E94610410920C0168
:100E100090911003943048F08091DE12882329F0DD
:100E2000109210030E949A3608C09F5F909310039F
:100E300004C00E9475360E94DD040E945336882348
:100E4000C1F78091460190914701019729F487E10C
:100E500093E061E070E004C087E193E06DE770E04B
:100E60000E94D32681EA90E09983888307C087E1B6
:100E700093E00E946C25892B09F0A3CF81E003C089
:100E80001982188283E0DF91CF910895CF93DF9389
:100E9000EC0181E090E0A0E0B0E08093790B9093CA
:100EA0007A0BA0937B0BB0937C0B84E290E0A0E0E4
:100EB000B0E08093810B9093820BA093830BB0934F
:100EC000840BCB01A0E0B0E08093850B9093860B60
:100ED000A093870BB093880B10928D0B10928E0B02
:100EE00010928F0B1092900B1092890B10928A0B1C
:100EF00010928B0B10928C0B1092910B1092920B04
:100F00001092930B1092940B1092950B1092960BDB
:100F10001092970B1092980B1092990B10929A0BBB
:100F200010929B0B10929C0B10929D0B10929E0B9B
:100F300010929F0B1092A00B1092A10B1092A20B7B
:100F40001092A30B1092A40B8C96A11DB11D80933F
:100F50007D0B90937E0BA0937F0BB093800B82E070
:100F60008093E9008091E8008F778093E80080917A
:100F7000E80085FFFCCFE9E7FBE081918093F10079
:100F80008BE0E53AF807C9F719C088818093F10032
:100F90008091E80085FD09C08091E8008F778093FB
:100FA000E8008091E80085FFFCCF442319F0779892
:100FB0009093770B21966150704001C09AE06115C3
:100FC000710519F78091E8008F778093E80081E040
:100FD000DF91CF9108955D988AE08093780B089512
:100FE00077988AE08093770B0895EF92FF921F9392
:100FF000CF93DF937C01FC01808191818C3E910530
:1010000009F465C0F1E084369F0709F423C1892BF8
:1010100009F028C18091780B882321F081508093BA
:10102000780B01C05D9A8091770B882321F0815065
:101030008093770B01C0779A8091650C9091660C34
:10104000029709F0F0C080913B01882351F088E2BB
:1010500093E069E170E00E945E250E94FA351092EB
:101060003B015F9A83E08093E9008091E80082FF72
:10107000DAC08091890C90918A0C892B09F0D3C039
:101080000E94E714209128033091290382179307C7
:1010900020F0EC01C21BD30B04C0C0912A03D091F5
:1010A0002B0388E293E00E943C25892BE1F481E048
:1010B00080931F0360912A0370912B036C1B7D0B9F
:1010C00080E293E00E94D3268CEE90E0BFC080E2E5
:1010D00093E00E946C25892B09F4C9C083E08093BA
:1010E000E90010921F0388E293E00E94532590913B
:1010F000F2009C3210F060E00BC08091E8008B7F22
:101100008093E8008091E8008F778093E80061E0A9
:10111000E9E7FBE08091F10081932BE0E53AF207EB
:10112000C9F7192F1C528091790B90917A0BA091DD
:101130007B0BB0917C0B0197A105B10559F0809113
:10114000E8008B7F8093E8008091E8008F778093A0
:10115000E80061E02091850B3091860B4091870B70
:101160005091880B211531054105510509F45BC0EB
:10117000662309F058C05D988AE08093780B6091EF
:10118000810B7091820B6452704016C08091F10007
:10119000115081F48091E8008B7F8093E80080916A
:1011A000E8008F778093E8008091E80082FFFCCF11
:1011B0001091F200615070406115710539F7B90165
:1011C000E1EDFCE01BC08091F100808321503040B4
:1011D000115099F42115310581F08091E8008B7F41
:1011E0008093E8008091E8008F778093E8008091F9
:1011F000E80082FFFCCF1091F200319621153105F5
:1012000011F78091E8008B7F8093E8008091E800DF
:101210008F778093E8006093890C70938A0C81ED3E
:101220009CE00E94393580914601909147010297D8
:1012300028F480E293E061E070E004C080E293E093
:101240006DE770E00E94D32684E691E0F701918378
:1012500080830DC080E293E00E946C25892B09F009
:10126000D9CE05C0F7011182108283E001C081E070
:10127000DF91CF911F91FF90EF90089581E08093CF
:101280002C0308958091E800877F8093E800909177
:101290002D03392FE0E01DC08091E80080FFFCCFD6
:1012A0002E2F5E2F505C0DC0432F4150251759F053
:1012B000E22FF0E0E754F44F80818093F1002F5F3C
:1012C000342F332389F78091E8008E7F8093E800E4
:1012D000E22F332339F08091E80082FFDDCF309395
:1012E0002D0302C010922D038091E80082FD13C0EF
:1012F000892F90E08F739070892B49F48091E800DA
:1013000080FFFCCF8091E8008E7F8093E800809181
:10131000E80082FFFCCF8091E8008B7F8093E8009B
:101320008091E8008F778093E80081E008959B0129
:10133000AC018091E80080FF47C080912D03882395
:1013400009F042C087E090E0A0E0B0E08093B90BE4
:101350009093BA0BA093BB0BB093BC0B84E190E0CD
:10136000A0E0B0E08093BD0B9093BE0BA093BF0BA9
:10137000B093C00B2093C10B3093C20B4093C30BAF
:101380005093C40BE9EBFBE081918093F1008BE07B
:10139000ED3CF807C9F78091E8008E7F8093E80064
:1013A0008091E80080FFFCCF8091E80082FFFCCFB5
:1013B0008091E8008B7F8093E8008091E8008F7730
:1013C0008093E80081E0089580E0089565FF02C001
:1013D00086E001C086E1809378010E94E1170895BC
:1013E000EF92FF920F931F93DF93CF93CDB7DEB7AA
:1013F00069970FB6F894DEBF0FBECDBF0091CD0B3D
:101400001091CE0B91ECE92E9BE0F92EE00EF11E2F
:10141000F70184819581A681B78183339105A10568
:10142000B10510F022E301C0282F30E0AE014F5F7C
:101430005F4F15C0E32FF0E0BA016E0F7F1FEE0F74
:10144000FF1FD7018D919C91E80FF91FE00FF11F4D
:10145000EF53F44F8081FB01808322503F5F1216CF
:101460004CF38091C50B9091C60BA091C70BB09126
:10147000C80B8B31F2E09F07F1E0AF07F0E0BF0748
:1014800009F43AC08C3122E0920721E0A20720E063
:10149000B207C8F48F30E1E09E07E1E0AE07E0E07C
:1014A000BE0709F499C08231F1E09F07F1E0AF0770
:1014B000F0E0BF0709F490C08E509140A140B040C9
:1014C00009F063C038C08130E1E09E07E1E0AE077B
:1014D000EDE0BE0709F44FC08230F1E09F07F1E074
:1014E000AF07FDE0BF0709F477C083509140A140EA
:1014F000B14009F04AC070C0CE01019663E476E0C5
:1015000047E050E00E942247892B09F065C0D701CF
:101510001C96ED91FC911D97EF53F44FE00FF11FD6
:1015200080812091D612803311F4277F01C028607A
:101530002093D61251C00F53144FF801608171816E
:101540008281938160932E0370932F0380933003E5
:1015500090933103611571058105910529F00E9471
:10156000E60982E090E002C081E090E09093660C92
:101570008093650C31C00F53144FD8018D919C910D
:10158000909345018093440127C085E090E0A0E05E
:10159000B0E88093B90B9093BA0BA093BB0BB093B8
:1015A000BC0B20E130E040E050E02093BD0B3093D5
:1015B000BE0B4093BF0B5093C00B81E090E0A0E0C6
:1015C000B0EC8093C50B9093C60BA093C70BB09360
:1015D000C80B20932D0322C085E090E0A0E0B0E886
:1015E0008093B90B9093BA0BA093BB0BB093BC0B39
:1015F00080E190E0A0E0B0E08093BD0B9093BE0B43
:10160000A093BF0BB093C00B1092C50B1092C60BEA
:101610001092C70B1092C80B80932D0369960FB6DA
:10162000F894DEBF0FBECDBFCF91DF911F910F9118
:10163000FF90EF900895E9EBFBE084E090E0A0E0FC
:10164000B0E88093B90B9093BA0BA093BB0BB09307
:10165000BC0B84E090E0A0E0B0E08093C90B9093D5
:10166000CA0BA093CB0BB093CC0B80E190E0A0E031
:10167000B0E08093CD0B9093CE0BA093CF0BB093A3
:10168000D00B8091C50B9091C60BA091C70BB09168
:10169000C80B853021E0920722E0A20720E0B207C4
:1016A00009F4DCC2863021E0920722E0A20720E0A4
:1016B000B20708F0BFC08D3021E0920721E0A207F9
:1016C00020E0B20709F4C8C18E3021E0920721E082
:1016D000A20720E0B20708F049C0863021E0920757
:1016E00021E0A20720E0B20709F4A2C1873021E07F
:1016F000920721E0A20720E0B207F8F4823021E04F
:10170000920721E0A20720E0B20709F4A7C28330C4
:1017100021E0920721E0A20720E0B20738F48150CF
:101720009140A140B04009F0A2C269C185509140EA
:10173000A140B04008F09BC291C28C3021E09207DA
:1017400021E0A20720E0B20708F081C18A3021E041
:10175000920721E0A20720E0B20708F073C187508A
:101760009140A140B04009F082C267C1863121E0BA
:10177000920721E0A20720E0B20709F48EC1873169
:1017800021E0920721E0A20720E0B20710F58F3098
:1017900021E0920721E0A20720E0B20709F482C10C
:1017A0008F3021E0920721E0A20720E0B20708F481
:1017B00066C1813121E0920721E0A20720E0B20753
:1017C00009F466C184519140A140B04009F04FC274
:1017D00045C2823021E0920722E0A20720E0B20752
:1017E00009F4FDC1833021E0920722E0A20720E046
:1017F000B20780F4823022E0920721E0A20720E0C5
:10180000B20709F42BC281509140A240B04009F0C8
:101810002EC2DCC1833021E0920722E0A20720E043
:10182000B20709F4EEC184509140A240B04009F0E3
:101830001EC2DEC1883021E0920721E0A2072DE020
:10184000B20709F4F0C0893021E0920721E0A20735
:101850002DE0B20708F06AC0853021E0920721E050
:10186000A20721E0B20709F4F9C1863021E092070E
:1018700021E0A20721E0B20740F5823021E0920783
:1018800021E0A20721E0B20709F438C1833021E04A
:10189000920721E0A20721E0B20738F4815091407D
:1018A000A140B14009F0E3C1FDC0833021E09207BF
:1018B00021E0A20721E0B20709F441C18450914020
:1018C000A140B14009F0D3C13FC1833021E092076C
:1018D00022E0A20721E0B20709F4C0C1843021E070
:1018E000920722E0A20721E0B20780F4813021E0D4
:1018F000920722E0A20721E0B20709F4AFC18250AB
:101900009140A240B14009F0B2C1A8C1813021E0AC
:10191000920721E0A2072DE0B20709F41AC1825014
:101920009140A140BD4009F0A2C136C18E3022E0F5
:10193000920721E0A2072DE0B20709F474C08F30AE
:1019400022E0920721E0A2072DE0B20740F58B319B
:1019500021E0920721E0A2072DE0B20709F463C05D
:101960008C3121E0920721E0A2072DE0B20738F484
:1019700088519140A140BD4009F079C154C08430E4
:1019800022E0920721E0A2072DE0B20709F466C128
:1019900086509240A140BD4009F069C112C180301B
:1019A00021E0920721E0A2072DEFB20709F43AC126
:1019B000813021E0920721E0A2072DEFB20778F4F1
:1019C000813122E0920721E0A2072DE0B20759F110
:1019D00087519240A140BD4009F049C124C08230E6
:1019E00021E0920721E0A2072DEFB20709F42DC1F3
:1019F00086509140A140BD4F09F039C12FC18CE8FC
:101A000090E0A0E0B0E08093C90B9093CA0BA09344
:101A1000CB0BB093CC0BCF01489667EB75E04CE84D
:101A200050E00E94194780E090E0A0E0B0E02BC1B8
:101A300080E095E0A0E0B0E0ECC084E690E0A0E0BB
:101A4000B0E0E7C086E690E0A0E0B0E0E2C08FEF53
:101A50009FEFAFEFB0E0DDC088E090E0A0E0B0E045
:101A60008093C90B9093CA0BA093CB0BB093CC0B74
:101A7000CF01489669E576E048E050E0D2CF80910A
:101A80002E0390912F03A0913003B0913103C1C078
:101A900084E195E0A0E0B0E0BCC080E090E1A0E08F
:101AA000B0E0B7C01092D50B1092D60B1092D70BA6
:101AB0001092D80B809141018093D10B809140010D
:101AC0008093D20B80913F018093D30B80913E0194
:101AD0008093D40B80913D018093D50B80913C0184
:101AE0008093D60B8091C90B9091CA0BA091CB0B20
:101AF000B091CC0B0296A11DB11D45C01092D50B23
:101B00001092D60B1092D70B1092D80B80914101F6
:101B10008093D10B809140018093D20B80913F0143
:101B20008093D30B80913E018093D40B80913D0133
:101B30008093D50B80913C018093D60B20C080E030
:101B400090E0A0E0BEE065C081E090E0A0E0B0E001
:101B500060C08091440190914501A0E0B0E0809385
:101B6000D10B9093D20BA093D30BB093D40B1092C4
:101B7000D50B1092D60B1092D70B1092D80B86E093
:101B800090E0A0E0B0E08093C90B9093CA0BA093C3
:101B9000CB0BB093CC0B47CF8DE090E0A0E0B0E052
:101BA0008093D10B9093D20BA093D30BB093D40B13
:101BB00085ED9BE06BE476E04DE050E00E9430471D
:101BC00032CF8CEE9FEFAFEFBFEF23C08091670C59
:101BD0009091680CA091690CB0916A0C1AC0809128
:101BE0006B0C90916C0CA0916D0CB0916E0C11C0AF
:101BF0008091730C9091740CA091750CB091760C3F
:101C000008C080916F0C9091700CA091710CB091F4
:101C1000720C8093D10B9093D20BA093D30BB09303
:101C2000D40B01CF86E090E0A0E0B0E08093C90B38
:101C30009093CA0BA093CB0BB093CC0B789686E015
:101C4000DF011D928A95E9F7EECE1092C90B109232
:101C5000CA0B1092CB0B1092CC0BE5CE1092D10B8D
:101C60001092D20B1092D30B1092D40BDCCE1092A8
:101C7000C90B1092CA0B1092CB0B1092CC0B81E0C7
:101C800090E0A0E0B0EC8093C50B9093C60BA093BE
:101C9000C70BB093C80B8091C90B9091CA0BA09150
:101CA000CB0BB091CC0B4896A11DB11D8093BD0B01
:101CB0009093BE0BA093BF0BB093C00B4897A109A4
:101CC000B10941F41092CD0B1092CE0B1092CF0BB4
:101CD0001092D00B8091BD0B80932D03089520911D
:101CE000E800277F2093E8009C018D3A910510F0D1
:101CF0002CEA30E08091E8008F7B8093E800E0E000
:101D000030C08091E8009091E80082FD02C096FF0B
:101D1000F8CF8091E80082FF1EC09E2F4E2F405CBE
:101D20008091F100E92FF0E0E754F44F80839F5F4A
:101D300021503040941719F02115310589F7809111
:101D4000E8008B7F8093E8008091E8008F77809394
:101D5000E800E92F06C08091E8008F7B8093E800BF
:101D600003C02115310569F68091E8008E7F8093CC
:101D7000E8008091B90B9091BA0BA091BB0BB09188
:101D8000BC0B84309105A105B10509F4A7C08530CD
:101D90009105A105B10558F482309105A105B10561
:101DA000C1F00397A105B10509F0F4C08DC08630DC
:101DB0009105A105B10509F497C086309105A105EB
:101DC000B10508F48EC00897A105B10509F0E2C07D
:101DD000BEC082E090E0A0E0B0E88093B90B9093A1
:101DE000BA0BA093BB0BB093BC0B24E330E040E0F4
:101DF00050E02093BD0B3093BE0B4093BF0B50932C
:101E0000C00B81E090E0A0E0B0E08093C90B90931C
:101E1000CA0BA093CB0BB093CC0B8093CD0B9093BC
:101E2000CE0BA093CF0BB093D00B1092C50B10929A
:101E3000C60B1092C70B1092C80B8093D10B9093D6
:101E4000D20BA093D30BB093D40B1092D50B10925E
:101E5000D60B1092D70B1092D80B8093D90B90937E
:101E6000DA0BA093DB0BB093DC0B8AE395E0A0E0E8
:101E7000B0E08093DD0B9093DE0BA093DF0BB0936B
:101E8000E00B83E090E0A0E0B0E08093E10B909362
:101E9000E20BA093E30BB093E40B1092E50B1092CE
:101EA000E60B1092E70B1092E80B1092E90B1092E0
:101EB000EA0B1092EB0B1092EC0B81E090E0909308
:101EC000660C8093650C40C05F9A5D987798769811
:101ED0008091E8008E7F8093E800FFCF0E941B0B6B
:101EE0005CC00E94F00959C01092660C1092650CFB
:101EF00086E090E0A0E0B0E88093B90B9093BA0B35
:101F0000A093BB0BB093BC0B20E130E040E050E06D
:101F10002093BD0B3093BE0B4093BF0B5093C00B6F
:101F20001092C10B1092C20B1092C30B1092C40BF3
:101F300081E090E0A0E0B0E08093C50B9093C60BE9
:101F4000A093C70BB093C80B20932D0326C088E045
:101F500090E0A0E0B0E88093B90B9093BA0BA09307
:101F6000BB0BB093BC0B80E190E0A0E0B0E08093AD
:101F7000BD0B9093BE0BA093BF0BB093C00B109200
:101F8000C50B1092C60B1092C70B1092C80B809312
:101F90002D0303C0779880E008958091E80080FFCA
:101FA000FCCF8091E80082FF0AC08091E8008B7F1F
:101FB0008093E8008091E8008F778093E80081E0CB
:101FC00080932C0308950F931F939091F1009093A9
:101FD0003A036091F1006630F9F0673068F46130DF
:101FE00009F405C1613008F471C1633009F439C1E5
:101FF000653009F0C0C1BFC0693009F4DEC06A3085
:1020000020F4683009F0B7C199C06A3009F49BC167
:102010006B3009F0B0C19EC1903809F08CC01092AD
:1020200032036091F1008091F1009091F100909164
:10203000F1001091F1000091F100813019F082302F
:1020400099F407C00E94CD3680937A0C0E94BB366B
:1020500006C00E94E13680937A0C0E94CF3690939E
:102060007C0C80937B0C05C00E946737882309F4A1
:1020700087C18091E800877F8093E80080917A0C87
:10208000811710F0002361F090E08F739070892B1E
:1020900021F481E08093320305C01092320302C024
:1020A00010937A0C20917B0C30917C0C40917A0C2F
:1020B00019C08091E80080FFFCCFF90190E00AC0D0
:1020C000542F5150903449F09F5F84918093F100D8
:1020D0003196452F9F01442399F78091E8008E7F28
:1020E0008093E800442359F08091E80082FFE1CF1B
:1020F00020937B0C30937C0C40937A0C06C0209389
:102100007B0C30937C0C10927A0C8091E80082FD5D
:102110000EC180913203813049F48091E80080FF44
:10212000FCCF8091E8008E7F8093E8008091E800EA
:1021300082FFFCCFFCC0892F66E009C19038C1F452
:102140008091E800877F8093E8008091790C8093EC
:10215000F1008091E8008E7F8093E8008091E80094
:102160008F778093E8008091E80082FFFCCFDFC08A
:10217000892F68E0ECC09923E9F49091E300809105
:10218000F1008F779078892B8093E3008091E800AD
:10219000877F8093E8008091E8008E7F8093E8003D
:1021A0008091E80080FFFCCF8091E30080688093FD
:1021B000E300F0C0892F65E0CAC09923A9F490918B
:1021C000F100923008F0DCC08091E800877F8093B6
:1021D000E8009093790C8091E8008E7F8093E8006E
:1021E000892F0E941238D6C0892F69E0B0C0933081
:1021F000A8F5992309F4C4C0913009F4C1C08091B5
:10220000F1009091F100882309F0BAC0E091F1004B
:10221000EF77E093E9008091EB0080FF51C0EE235F
:10222000B1F08091EB0080618093EB0081E090E061
:102230000E2E02C0880F991F0A94E2F78093EA00DD
:102240001092EA008091EB0088608093EB0010927E
:10225000E900F0E0ED5CFC4F108229C0892F61E0BD
:1022600076C0933080F5913009F48AC0923009F03D
:1022700091C08091F1009091F100882309F080C015
:10228000E091F100EF7709F47BC0E093E9008091E1
:10229000EB0080FF15C08091EB0080628093EB0023
:1022A0001092E900F0E0ED5CFC4F81E080838091CA
:1022B000E800877F8093E8008091E8008E7F68C007
:1022C0001092E9005DC0892F63E041C0892F8058DA
:1022D0008330B0F58091F1008091F100E091F10040
:1022E000913829F0923859F0903809F049C080911E
:1022F000E800877F8093E8001092F1000DC0809184
:10230000E800877F8093E800F0E0EF77F070ED5C05
:10231000FC4F80818093F1001092F1008091E800E1
:102320008E7F8093E8008091E80082FFFCCF80914F
:10233000E8008B7F8093E8008091E8008F7728C0C9
:10234000892F60E004C09138D9F0892F6AE00E949B
:10235000933820C09130F1F48091E800877F80931A
:10236000E8008091E8008E7F8093E8008091E8008B
:1023700080FFFCCF0FC0892F0E949338882351F42F
:102380008091EB0080628093EB008091E800877F72
:102390008093E8001F910F910895789483B7817F0F
:1023A000846083BF83B7816083BF889583B78E7F46
:1023B00083BF08958EE089BD09B400FEFDCF8091F2
:1023C000D8008F7D8093D8008091D8008160809361
:1023D000D8008091E20088608093E2000E943B3741
:1023E0008091E0008E7F8093E00008951F93CF934B
:1023F000DF93EC01162F623891F580911F0388233B
:1024000051F51092E9008091E80083FF02C00E941C
:10241000E30F80912C038823F1F091E09093E90081
:102420008091E80085FF17C09093F1001092F100B1
:102430001092F1001092F1001092F1001092F10050
:102440001092F1001092F1008091E8008F77809354
:10245000E80010922C0384E591E00E94F724888123
:102460009981009729F08551914009F056C051C0DB
:102470008091D70081608093D7008091D7008F7BB7
:102480008093D7008091D70080688093D70078949C
:102490008091D8008F768093D8008091D800806991
:1024A0008093D8008091D8008F7B8093D800809152
:1024B000D80081608093D800789484E591E00E94F0
:1024C000F7248091D90080FF09C080917D0C88237A
:1024D00029F481E080937D0C0E94DA1180913B0306
:1024E00090913C0390FF10C080913B0390913C037E
:1024F0009E7F90933C0380933B0381E08093EA00AE
:102500001092EA001092790C85E191E0998388831A
:1025100002C01F32B1F281E003C01982188283E049
:10252000DF91CF911F9108951F920F920FB60F92D6
:102530000BB60F9211242F933F934F935F936F939A
:102540007F938F939F93AF93BF93EF93FF9384E514
:1025500091E06FE240E050E00E9497248091DA0021
:1025600080FF31C08091D80080FF2DC08EEF809316
:10257000DA008091D90080FF19C081E080937D0C42
:1025800080913B0390913C03826090933C03809345
:102590003B038091E20088608093E2000E94DA11A0
:1025A0008091E0008E7F8093E0000DC010927D0C42
:1025B0001092790C80913B0390913C03846090933E
:1025C0003C0380933B038091E10082FF07C0809130
:1025D000E20082FF03C08BEF8093E1008091E10075
:1025E00080FF29C08091E20080FF25C08EEF80939C
:1025F000E1008091E20080618093E2008FEE8093A1
:10260000E1008091D80080628093D80080913B03E4
:1026100090913C03806290933C0380933B037894B9
:1026200083B7817F846083BF83B7816083BF8895D0
:1026300083B78E7F83BF8091E10084FF1AC08091B1
:10264000E20084FF16C08091D8008F7D8093D8006F
:102650008FEE8093E1008091E2008F7E8093E20014
:1026600080913B0390913C03806490933C03809362
:102670003B038091E10085FF1AC08091E20085FF55
:1026800016C08091E2008F7E8093E2008FED8093F0
:10269000E1008091E2008F7D8093E20080913B0316
:1026A00090913C03806890933C0380933B0380911E
:1026B000E10083FF12C08091E20083FF0EC087EF2C
:1026C0008093E1000E943B3780913B0390913C0353
:1026D000916090933C0380933B03FF91EF91BF91F6
:1026E000AF919F918F917F916F915F914F913F91AA
:1026F0002F910F900BBE0F900FBE0F901F9018954B
:102700001F9381E08093E90011E00AC01092E90074
:102710008091E80083FF02C00E94E30F1093E9005C
:102720008091EB0085FDF2CF82E08093E90012E01A
:102730000AC01092E9008091E80083FF02C00E9465
:10274000E30F1093E9008091EB0085FDF2CF81E06B
:102750008093E9008091E80085FFFCCF85E58093B8
:10276000F10093E59093F10082E48093F10090935F
:10277000F10080913E038093F10080913F038093AC
:10278000F100809140038093F10080914103809398
:10279000F1008091E4128093F1008091E312809324
:1027A000F1008091E2128093F1008091E112809318
:1027B000F1008091F5128093F1008091E8008F770D
:1027C0008093E8001F91089582E08093E9002091B2
:1027D000F1008091F100833519F490E0253509F07E
:1027E00091E08091F100823409F091E08091F10054
:1027F000833409F091E08091F10080933E03809151
:10280000F10080933F038091F10080934003809119
:10281000F100809341038091F1008093E112809157
:10282000F1008093E2128091F1008093E312809195
:10283000F1008093E4128091F1008823B9F021E047
:1028400020933D03992331F18091E8008B7F8093A1
:10285000E8008091E8008F778093E8002093E900FA
:102860008091EB0080628093EB00089510923D030D
:10287000992381F08091EB0080628093EB0080913E
:10288000E8008B7F8093E8008091E8008F77809349
:10289000E80008958091F10080937E0C8091E01211
:1028A000882321F40E946F3D80937E0C8091F1007B
:1028B000E5EEF2E18091F100819382E1E53FF807D6
:1028C000C9F78091E8008B7F8093E8008091E80051
:1028D0008F778093E80080913D03813011F48093DD
:1028E000E9000E941D3D813089F08091E1129091B4
:1028F000E212A091E312B091E4120097A105B10594
:1029000029F08091EB0080628093EB000895CF93D3
:10291000DF93EC0188819981009721F08638910539
:10292000A1F52BC08091460190914701029779F45F
:102930008091790C882359F082E08093E90080919E
:10294000E80082FF04C00E94E4130E94801380917B
:10295000460190914701029729F482E493E061E0F7
:1029600070E004C082E493E06DE770E00E94D3263B
:1029700086E890E09983888306C082E493E00E9411
:102980006C25892B79F681E003C01982188283E0D7
:10299000DF91CF910895F8941092B60016BC8EE3A3
:1029A00087BD92E094BD85E085BD85B385BB9093DE
:1029B0006E0010924B0310924A0380914A0390914B
:1029C0004B0390934D0380934C037894089520918A
:1029D0004A0330914B0380914A0390914B0328178F
:1029E0003907A9F7C901089507C022E330E00000C4
:1029F00021503040E1F701970097B9F70895BC01E5
:102A000040914A0350914B0380914A0390914B03AC
:102A100048175907A9F720914A0330914B03809139
:102A20004A0390914B0328173907A9F7241B350B4C
:102A30002617370780F30895089520914E033091AB
:102A40004F03409150035091510380914E03909158
:102A50004F03A0915003B0915103281739074A073B
:102A60005B0759F7B901CA0108951F920F920FB67B
:102A70000F920BB60F9211242F933F934F935F93B6
:102A80006F937F938F939F93AF93BF93EF93FF9336
:102A900080914A0390914B03019690934B0380934E
:102AA0004A0380914C0390914D03019690934D03FE
:102AB00080934C0380914C0390914D038D37910589
:102AC000B9F410924D0310924C0380914E039091F3
:102AD0004F03A0915003B09151030196A11DB11D68
:102AE00080934E0390934F03A0935003B0935103F0
:102AF0000E948425892B11F00E940326FF91EF91FB
:102B0000BF91AF919F918F917F916F915F914F9105
:102B10003F912F910F900BBE0F900FBE0F901F9003
:102B200018958BE593E0089580915A03089580915C
:102B30005803089580E01C9981E008952D982C9801
:102B40008CE090E00197F1F72D9A0895DF92EF92D3
:102B5000FF920F931F93DF93CF9300D00F92CDB7C7
:102B6000DEB70091660080E88093660010927000E6
:102B700010926F008091B60080628093B6008091C1
:102B8000B6008B71E1F781E08093B1008FB7898344
:102B9000F89410E8DD24D39480E8E82EFF24FA941A
:102BA000D09281008091B6008B71E1F7E092B20083
:102BB0001092850010928400F7BAB89BFECF8091E6
:102BC0008400909185009B838A83109281006A81A2
:102BD0007B8180E090E00E942C4420E03FEE47EEB5
:102BE00056E40E94FC43882324F4809166008F5FA2
:102BF00013C06A817B8180E090E00E942C4420E831
:102C00003CE240E057E40E94CC43181614F081E007
:102C100006C08091660081508093660080E011506C
:102C200021F0882309F4BCCF04C0882311F4009359
:102C300066001092B1008091B6008F7D8093B6003F
:102C400089818FBF0F900F900F90CF91DF911F91CF
:102C50000F91FF90EF90DF900895282F8EE268E0AB
:102C600043E00E94E11B0895882329F085E060E895
:102C700047E021E004C085E060E847E020E00E94F2
:102C8000E11B08952C988CE090E00197F1F782E029
:102C90006FE140E023E00E94E11B82E090E00197B9
:102CA000F1F708951F93162F603118F022E430E0F9
:102CB0001AC01C9B03C024E430E015C0882329F00F
:102CC00081E160E144E021E004C081E160E144E0B1
:102CD00020E00E94E11B81E16FE040E0212F0E9493
:102CE000E11B20E430E0C9011F9108951F93282FB4
:102CF000162F8330A8F4603198F41C9B03C024E4A1
:102D000030E010C088E060E645E00E94E11B89E009
:102D10006FE040E0212F0E94E11B20E430E002C080
:102D200022E430E0C9011F910895282F803118F066
:102D300022E430E00CC01C9B03C024E430E007C058
:102D400085E06FE040E00E94E11B20E430E0C90133
:102D500008950F931F93082F162F1C9B03C024E484
:102D600030E02BC08CE260EF44E020E00E94E11BE9
:102D7000212F30E02873307093E0359527959A9590
:102D8000E1F78CE26EE041E00E94E11B212F2295E9
:102D90002695269523708EE260EC46E00E94E11BAA
:102DA0008DE2602F0E94B31B17708EE267E040E057
:102DB000212F0E94E11B20E430E0C9011F910F91F7
:102DC0000895AF92BF92CF92DF92EF92FF920F934E
:102DD0001F938C017C010894E11CF11C84E2F80132
:102DE00060810E94B31B67010894C11CD11C85E25D
:102DF000F80161810E94B31B56010894A11CB11C0B
:102E000086E2F70161810E94B31B75010894E11C01
:102E1000F11C87E2F60161810E94B31B87010F5FFD
:102E20001F4F88E2F50161810E94B31B89E2F7011F
:102E300061810E94B31B8AE2F80161810E94B31B89
:102E40008BE20F5F1F4FF80161810E94B31B1F913E
:102E50000F91FF90EF90DF90CF90BF90AF900895CB
:102E60001F93682F192F80E20E94B31B81E2612F0C
:102E70000E94B31B1F9108951F93682F192F82E2A0
:102E80000E94B31B83E2612F0E94B31B1F91089520
:102E9000EF92FF920F931F937C0184E20E94981B94
:102EA000F70181938F0185E20E94981BF7018183CE
:102EB00078010894E11CF11C86E20E94981BF8013D
:102EC000818387010F5F1F4F87E20E94981BF701E4
:102ED000818378010894E11CF11C88E20E94981B10
:102EE000F801818387010F5F1F4F89E20E94981BC1
:102EF000F70181838AE20E94981BF80181838BE2AB
:102F00000E94981B0F5F1F4FF80181831F910F9143
:102F1000FF90EF9008951F9381E20E94981B182F55
:102F200081E20E94981B512F40E0282F30E0242B93
:102F3000352BC9011F9108951F9383E20E94981BAE
:102F4000182F82E20E94981B512F40E0282F30E07A
:102F5000242B352BC9011F9108958EE268E043E0D0
:102F60000E94CE1B089581E06FE140E00E94CE1BDD
:102F700008951C9904C020E430E0C90108952C98FC
:102F800080EE96E00197F1F781E06FE140E00E946A
:102F9000CE1B883081F323E430E0EFCF1C990DC0C5
:102FA0000E94421681E06FE140E00E94CE1B883013
:102FB00019F023E430E003C02C9A20E430E0C9018A
:102FC00008950F931F93082F883059F0863049F0E9
:102FD000893039F0863129F0893119F022E430E066
:102FE00056C01C9B03C024E430E051C081E06FE177
:102FF00040E00E94CE1B182F81518230B8F311306F
:10300000A9F3123099F3011709F43FC0083019F4FD
:103010000E94421626C0093139F4163199F482E033
:103020006FE140E029E008C0063161F4193151F444
:1030300082E06FE140E026E00E94E11B82E090E048
:103040000197F1F782E06FE140E0202F0E94E11B41
:10305000183019F488E691E002C082E090E0019710
:10306000F1F781E06FE140E00E94CE1B801719F07C
:1030700023E430E00CC0063011F0063121F481E089
:103080008093590302C01092590320E430E0C90133
:103090001F910F91089581E06FE140E00E94CE1BE7
:1030A0008850823018F024E430E016C088E160E8EF
:1030B00047E021E00E94E11B82E390E00197F1F7F5
:1030C00088E160E847E00E94CE1B882319F420E4E1
:1030D00030E002C023E430E0C901089583E067E0F6
:1030E00040E00E94CE1B08950F931F93082F162FC8
:1030F000663018F022E430E01CC083E067E040E076
:103100000E94CE1B811799F0002329F483E068E028
:1031100043E021E004C083E068E043E020E00E9457
:10312000E11B83E067E040E0212F0E94E11B20E4E7
:1031300030E0C9011F910F910895DF92EF92FF9245
:103140000F931F93D0906600F89481E061E00E9495
:103150007418E090B100F09081000091800010920E
:10316000B100109281001092800020E030E04FEF1B
:1031700063E056E046BB47BB1092B2001092850058
:10318000109284006093B10050938100B89BFECFF1
:10319000109281001092B10080918400909185007E
:1031A00073E08A3F970720F480916600815008C041
:1031B0008650944010F411E00CC0809166008F5F3F
:1031C000809366002F5F3F4F83E0283E380791F6DB
:1031D00010E081E060E00E947418E092B100F0928B
:1031E000810000938000112311F4D0926600812F9A
:1031F0001F910F91FF90EF90DF90089581E160E2C1
:1032000045E00E94CE1B882319F02BE430E002C079
:103210002AE430E0C901089581E160E144E00E94C0
:10322000CE1B089581E16FE040E00E94CE1B08951F
:10323000CF93DF93EC0181E06FE140E00E94CE1B71
:10324000863029F0813019F024E430E008C086E0AF
:103250006FE140E00E94CE1B888320E430E0C9018A
:10326000DF91CF91089589E06FE040E00E94CE1B8E
:10327000089588E060E645E00E94CE1B089585E051
:103280006FE040E00E94CE1B089588E06FE140E0CF
:103290000E94CE1B08951F93182F8B50803118F079
:1032A00022E430E02BC01C9B03C024E430E026C0A5
:1032B00088E06FE140E00E94CE1B8117E9F088E0D2
:1032C0006FE140E0212F0E94E11B81E06FE140E0CF
:1032D0000E94CE1B863011F0893021F48CE291E0FF
:1032E0000197F1F788E06FE140E00E94CE1B811763
:1032F00019F023E430E002C020E430E0C9011F915E
:103300000895DF92EF92FF920F931F937B018C0140
:10331000D42E86E06FE140E00E94CE1B80935803DC
:10332000E0915203F0915303309721F0C801B701A7
:103330004D2D09951F910F91FF90EF90DF9008950B
:103340001F93CF93DF93182FEB0187FF03C022E475
:1033500030E01FC081E06FE140E00E94CE1B823070
:10336000B1F081E06FE140E00E94CE1B823179F044
:1033700088E00E94E11789E10E94E1172C9A2C98BD
:10338000CE01612F0E94BC1C20E430E002C024E486
:1033900030E0C901DF91CF911F91089581E06FE185
:1033A00040E00E94CE1B893019F024E430E029C0AF
:1033B0008BE160E847E021E00E94E11B8AE160E8E0
:1033C00047E021E00E94E11B0E94881B8CE291E013
:1033D0000197F1F70E94851B882389F08BE160E853
:1033E00047E00E94CE1B882351F48AE160E847E061
:1033F0000E94CE1B882319F420E430E002C023E4AD
:1034000030E0C9010895CF92DF92EF92FF920F93BF
:103410001F93CF93DF938B017A016901ECEFF3E007
:103420003197F1F7882311F00E94A6150E94D01A57
:103430002D982C988CE090E00197F1F72D9A82E07E
:103440006FE140E023E00E94E11B8CEF93E00197E5
:10345000F1F781E06FE140E00E94CE1B883019F067
:10346000C3E4D0E014C08DE10E94981B81508230EB
:1034700060F48EE10E94981B8F3139F48EE06CE08D
:103480000E94B31BC0E4D0E002C0C1E4D0E01093BE
:10349000530300935203F0925503E092540381E8E2
:1034A00099E10E94611B85E69AE10E94381BD09247
:1034B0005703C0925603CE01DF91CF911F910F9118
:1034C000FF90EF90DF90CF900895DF93CF9300D0DF
:1034D00000D00F92CDB7DEB79B01AC01E091540351
:1034E000F0915503309711F0099552C0809159031E
:1034F0008823C1F02093EF033093F0034093F1034E
:103500005093F203809158038093EE038AE593E091
:1035100060E070E00E94161C8AE593E06CED73E0B9
:103520000E94EA1D80915903882391F588E00E944A
:10353000E117809178010E94E1171B821A821D8297
:103540001C8282E060EE45E00E94CE1B8983898167
:10355000833059F0843018F4823058F403C0853039
:1035600041F403C081E190E002C082E190E09B83DE
:103570008A838A819B81892B21F0CE0102960E9449
:1035800014204C815D818CE991E06A810E9497242E
:103590000F900F900F900F900F90CF91DF910895A3
:1035A000DF93CF930F92CDB7DEB71092F503109251
:1035B000F4038FB78983F8941092F6031092F703FF
:1035C0001092F9031092F8031092FB031092FA0381
:1035D00089818FBF249A259A84B1876084B985B187
:1035E000836085B980E58CBD81E08DBD83E48093E7
:1035F0008100B59AEFE6F0E0808181608083808170
:10360000806280830F90CF91DF910895DF93CF93F5
:103610000F92CDB7DEB78FB78983F8941092F60377
:103620001092F7031092F9031092F8031092FB0323
:103630001092FA0389818FBF0F90CF91DF91089587
:103640008091F6030895DF93CF930F92CDB7DEB745
:103650008FB78983F8941092F60389818FBF0F90FA
:10366000CF91DF9108958091FA039091FB03089523
:10367000DF93CF930F92CDB7DEB72FB72983F8949E
:103680009093FB038093FA0389818FBF0F90CF91B2
:10369000DF910895DF93CF930F92CDB7DEB78FB749
:1036A0008983F8941092FB031092FA0389818FBFEB
:1036B0000F90CF91DF9108958091F8039091F903D5
:1036C0000895DF93CF930F92CDB7DEB72FB729833D
:1036D000F8949093F9038093F80389818FBF0F903A
:1036E000CF91DF910895DF93CF930F92CDB7DEB7DF
:1036F0008FB78983F8941092F9031092F8038981A7
:103700008FBF0F90CF91DF9108958091F7030895B7
:10371000DF93CF930F92CDB7DEB78FB78983F8943D
:103720001092F70389818FBF0F90CF91DF91089599
:10373000DF93CF930F92CDB7DEB780689FB79983A1
:10374000F89428988EBD0DB407FEFDCF8EB58EBDC2
:103750000DB407FEFDCF8EB5289A99819FBF0F90BB
:10376000CF91DF910895DF93CF930F92CDB7DEB75E
:10377000806C9FB79983F89428988EBD0DB407FE8E
:10378000FDCF8EB56EBD0DB407FEFDCF8EB5289A68
:1037900089818FBF0F90CF91DF910895FF920F9392
:1037A0001F93062FF42E0E94981B082310E002C0DE
:1037B00015950795FA94E2F7802F1F910F91FF90CE
:1037C0000895EF92FF920F931F93DF93CF930F9281
:1037D000CDB7DEB7182F062FE42EF22E0E94981BCD
:1037E000282F106C8FB78983F89428981EBD0DB4CC
:1037F00007FEFDCF8EB58F2D90E002C0880F991F78
:10380000EA94E2F7802300950223802B8EBD0DB44D
:1038100007FEFDCF8EB5289A89818FBF0F90CF917B
:10382000DF911F910F91FF90EF9008958F929F92DB
:10383000AF92BF92CF92DF92EF92FF920F931F93BE
:10384000DF93CF930F92CDB7DEB78C014B0100977A
:1038500021F46115710509F481C08FB78983F8944B
:10386000289880E28EBD0DB407FEFDCF8EB58EBDCB
:103870000DB407FEFDCFEEB48E2D83508D3708F0CA
:1038800060C00115110539F068010894C11CD11CF4
:10389000F801E08206C08E2D90E0F4010995CC2459
:1038A000DD24EEBC0DB407FEFDCFAA24BB24FEB47C
:1038B0001EBC0115110521F0F601F1926F0104C043
:1038C0008F2D90E0F4010995C5018F25082E829572
:1038D000807F8025092E982F82958F7008268695E7
:1038E00098278927880F880F880F80255C010DB4E1
:1038F00007FEFDCFEA94D9F60115110541F08EB50A
:1039000000581F4FF80180830058104004C08EB546
:1039100090E0F4010995289A0115110549F0F80184
:10392000EF57FF4F1082AB28B9F481E0808314C0B9
:1039300080E090E0AB2811F081E090E0F40109957F
:103940000BC0289A0115110539F0F80110820058B2
:103950001F4FF8011192108289818FBF0F90CF9174
:10396000DF911F910F91FF90EF90DF90CF90BF906C
:10397000AF909F908F900895DF93CF930F92CDB724
:10398000DEB7FC016F778FB78983F894289880E6BB
:103990008EBD0DB407FEFDCF8EB56EBD0DB407FE16
:1039A000FDCF8EB581918EBD61500DB407FEFDCF68
:1039B0008EB56623B9F7289A89818FBF0F90CF9172
:1039C000DF910895DF93CF930F92CDB7DEB7982F95
:1039D000FA018FB78983F89428981EBC0DB407FEAE
:1039E000FDCF8EB59EBD0DB407FEFDCF8EB51EBCBE
:1039F0000DB407FEFDCF8EB58083615011F0319676
:103A0000F6CF289A89818FBF0F90CF91DF910895CB
:103A1000DF93CF930F92CDB7DEB7982FFA018FB710
:103A20008983F894289880E48EBD0DB407FEFDCFFD
:103A30008EB59EBD0DB407FEFDCF8EB581918EBDB6
:103A40000DB407FEFDCF8EB56150C1F7289A89816C
:103A50008FBF0F90CF91DF9108951F920F920FB6F5
:103A60000F920BB60F9211240F931F932F933F9336
:103A70004F935F936F937F938F939F93AF93BF9376
:103A8000EF93FF93DF93CF930F92CDB7DEB7809183
:103A9000F4039091F503A0E0B0E09C01112700270A
:103AA0008091840090918500A0E0B0E0082B192B54
:103AB0002A2B3B2B28988FE88EBD36952795179596
:103AC00007950DB407FEFDCF8EB58EBD0DB407FE74
:103AD000FDCF9EB5289A92FF18C0E091F803F091AF
:103AE000F903309709F447C0289880E28EBD0DB4E1
:103AF00007FEFDCF8EB58EBD0DB407FEFDCF4EB5D2
:103B0000289AC901B801099536C093FF0AC0E0910F
:103B1000FA03F091FB03309771F1C901B8010995DF
:103B20002AC096FD28C091FD26C090FF06C0809156
:103B3000F7038F5F8093F7031EC097FF1CC08EE0D2
:103B40000E94981B982F8FB78983F89428988EEC41
:103B50008EBD0DB407FEFDCF8EB59F779EBD0DB413
:103B600007FEFDCF8EB5289A89818FBF8091F6031D
:103B70008F5F8093F6030F90CF91DF91FF91EF91CC
:103B8000BF91AF919F918F917F916F915F914F9175
:103B90003F912F911F910F910F900BBE0F900FBE71
:103BA0000F901F9018951F920F920FB60F9211242D
:103BB0008F939F938091F4039091F50301969093D6
:103BC000F5038093F4039F918F910F900FBE0F9098
:103BD0001F9018950F931F93DF93CF93CDB7DEB748
:103BE00028970FB6F894DEBF0FBECDBF8C01DB0166
:103BF00057968C91579781FF19C08091FC038823B9
:103C000089F485E190E09A8389831C821B82CE012E
:103C100001960E9414204B815C818CE991E06981BE
:103C20000E94972481E08093FC039BC0A8014F5F12
:103C30005F4F11965C934E930D5F1F4F13961C932D
:103C40000E93129703501040F801818187708230E3
:103C500021F450961C92509765C098012C5F3F4FFD
:103C6000882331F115963C932E93149798012A5F7F
:103C70003F4F17961C921E921697FA0181818695E6
:103C800086958E5F8370823098F417963C932E93BE
:103C900016978181869586958370823021F49801EC
:103CA000285F3F4F05C0833019F49801225F3F4FD2
:103CB00019961C921E921897F801818186FD07C003
:103CC00019963C932E9318972E5F3F4F08C0149679
:103CD0008D919C91159719969C938E9318971B968E
:103CE0003C932E931A97FA01818182958695869549
:103CF0008370823019F42E5F3F4F04C0833011F47B
:103D0000285F3F4F1D961C921E921C97F8018081E0
:103D10008250840F821B50968C9350971F963C9331
:103D20002E931E9700581F4FF801819151968C9346
:103D300051978081817057962C9157972E7F282B11
:103D400080E190E09E838D83B887AF832260579691
:103D50002C93CE0105960E9414208CE991E00E94DC
:103D6000F72428960FB6F894DEBF0FBECDBFCF91D3
:103D7000DF911F910F910895CF92DF92FF920F93E1
:103D80001F93DF93CF9300D000D00F92CDB7DEB753
:103D90008C016B01FE01319685E0DF011D928A9551
:103DA000E9F7F801218126952695237011F082E02C
:103DB0008983D80111969C919295969596959370CA
:103DC00011F082E08B83291721F4F801808180644F
:103DD0008083D8018C9186FD1B82F80181818695B4
:103DE0008695837090E08230910519F0039729F44D
:103DF00002C082E001C088E08A83D80111968C91CC
:103E0000829586958695837090E08230910519F0B1
:103E1000039729F402C082E001C088E08C83F80196
:103E2000808183FF1DC087898695869586958370DE
:103E300090E08130910571F0823091051CF4892B5E
:103E400039F00EC08230910539F0039749F406C06D
:103E500085E005C086E003C08AE001C08EE08D8366
:103E6000D8018D919C9111979093FE038093FD034F
:103E700012968C918093FF038981823019F093E030
:103E8000F92E09C0F80183819481909301048093F5
:103E9000000485E0F82E8A81823019F08830A1F57F
:103EA0000DC0EF2DF0E0E350FC4FD80115968D9139
:103EB0009C91169791838083B2E025C0EF2DF0E0AE
:103EC000E350FC4FD80115968C9115978083169678
:103ED0008C911697818317968C91179782831896E9
:103EE0008C911897838319968C91199784831A96CD
:103EF0008C911A9785831B968C911B9786831C96B1
:103F00008C918783B8E0FB0E8B81823069F4EF2DB2
:103F1000F0E0E350FC4FD8011D968D919C911E97C7
:103F200091838083B2E0FB0E8C81823019F088305F
:103F3000A1F50DC0EF2DF0E0E350FC4FD8011F9626
:103F40008D919C91509791838083B2E025C0EF2D95
:103F5000F0E0E350FC4FD8011F968C911F978083AF
:103F600050968C915097818351968C915197828372
:103F700052968C915297838353968C915397848356
:103F800054968C915497858355968C91559786833A
:103F900056968C918783B8E0FB0EED81EE2379F085
:103FA0002F2D30E023503C4FA801495E5F4FC901DF
:103FB000BA014E2F50E00E944C478D81F80E2F2DF4
:103FC00030E023503C4FF80147A165A176A1C9011B
:103FD00050E00E944C47D80197968C918E5F8F0DD0
:103FE000F60182838DEF93E0918380830F900F9091
:103FF0000F900F900F90CF91DF911F910F91FF9035
:10400000DF90CF9008959C01F999FECF32BD21BD7C
:10401000F89A80B5089520E09091910480919204DF
:10402000981321E0822F0895CF93DF93EC01409104
:104030009104E42FF0E0CF0101966AE070E00E9465
:10404000634A2091920430E082179307A9F0888197
:104050009981AA81BB81EE0FFF1FEE0FFF1FEF5664
:10406000FB4F82839383A483B583842F8F5F8A3031
:1040700008F080E080939104DF91CF910895DF9361
:10408000CF930F92CDB7DEB78091920489832981B7
:1040900089818F5F898389818A3008F019828981BB
:1040A0008093920430E0220F331F220F331F2D56CE
:1040B0003B4FC9010F90CF91DF9108959093800CF1
:1040C00080937F0C089581E090E0089581E090E076
:1040D000089589E791E0089580918F04909190046C
:1040E000089581E894E00895AC01615020E00CC08F
:1040F000DA01A20FB11D9C91FA01E60FF11D80813A
:104100008C93908361502F5F261790F308950F933F
:104110001F93DF93CF930F92CDB7DEB78823E9F1DA
:104120000FEF1FEF10930B1300930A130E94EB463F
:1041300060E071E00E94634A80934D138DEC9BEA2E
:1041400090933913809338139093FF128093FE124B
:1041500010930913009308138FB78983F89480E0B4
:1041600093E160E070E048E050E023E030E20E943C
:10417000674720E037E0A22FB0E0A050BD4E9C91F1
:10418000E32FE21BF0E0E050FD4E80818C939083A2
:104190002F5F243081F789818FBF0F90CF91DF91FE
:1041A0001F910F910895CF92DF92EF92FF920F939C
:1041B0001F93DF93CF93CDB7DEB7AB970FB6F894CD
:1041C000DEBF0FBECDBF80EB96E30197F1F782E033
:1041D0000E94C7418093FD128C81807E81608C8318
:1041E00082E10E94C74120E0892B09F021E022955D
:1041F000220F207E8C818F79822B8C839D819F7CE6
:1042000080914D138E838F5F80934D13906C9D83AF
:10421000E0911613F0911713099598878F8385E124
:104220000E94D04164E072E00E942343892B59F040
:104230008D81837F88608D838FEF9FEF98878F8339
:104240009A87898722C085E10E94D041DE011996B4
:10425000FC0188E001900D928150E1F7AE01475FCB
:104260005F4F20E037E0DA01A20FB11D9C91832F50
:10427000821BFA01E80FF11D80818C9390832F5FE0
:10428000243089F78D818C608D83E0911A13F09131
:104290001B1309959A8B898BE0912213F0912313BC
:1042A00009952B8B3C8B4D8B5E8B6F8B788F898F19
:1042B0009A8F0E94A6418BA70E9478419AA789A74E
:1042C00074E0E72EF12CEC0EFD1EC7018E010F5F8E
:1042D0001F4FB8010E94BC1EC701B8010E949B324B
:1042E00003E068ECE62EF12C50E2C52E5EE4D52EFC
:1042F00069817A818B810E94A0198034910519F41B
:1043000021E030E020C084349105D9F4033021F459
:10431000C6010197F1F713C0023041F484EF91E038
:10432000F7013197F1F70197D9F709C0013039F456
:1043300080ED97E0F7013197F1F70197D9F7015038
:10434000B9F620E030E0C901AB960FB6F894DEBFB5
:104350000FBECDBFCF91DF911F910F91FF90EF90D6
:10436000DF90CF90089580917F0490918004892BF5
:1043700009F467C00E940942E0918F04F091900413
:1043800060898685978570E00E94EC42E0918F04F9
:10439000F0919004808990E00E947341E0918F0435
:1043A000F0919004ABEBB4E026813781C901FC01A8
:1043B00088E001900D928150E1F7E0918F04F09137
:1043C0009004A3ECB4E022853385C901FC0188E0A8
:1043D00001900D928150E1F720E037E0A22FB0E08C
:1043E000A554BB4F9C91E32FE21BF0E0E554FB4F3B
:1043F00080818C9390832F5F243081F720E037E019
:10440000A22FB0E0AD53BB4F9C91E32FE21BF0E035
:10441000ED53FB4F80818C9390832F5F243081F785
:1044200085E16BEB74E00E94DB4184E163EC74E0B6
:104430000E94DB41E0917F04F091800481E894E0E8
:10444000099508950E940942E0918F04F09190042B
:1044500060898685978570E00E94EC42E0918F0428
:10446000F0919004808990E00E947341E0918F0464
:10447000F0919004ABEBB4E026813781C901FC01D7
:1044800088E001900D928150E1F7E0918F04F09166
:104490009004A3ECB4E022853385C901FC0188E0D7
:1044A00001900D928150E1F720E037E0A22FB0E0BB
:1044B000A554BB4F9C91E32FE21BF0E0E554FB4F6A
:1044C00080818C9390832F5F243081F720E037E048
:1044D000A22FB0E0AD53BB4F9C91E32FE21BF0E065
:1044E000ED53FB4F80818C9390832F5F243081F7B5
:1044F00085E16BEB74E00E94DB4184E163EC74E0E6
:104500000E94DB41E0917F0CF091800C81E894E007
:1045100009950895DF93CF930F92CDB7DEB79091B1
:104520009204809191048917A1F199838981E82FE0
:10453000F0E0EE0FFF1FEE0FFF1FED56FB4F8981DE
:104540008F5F898389818A3008F0198289818093FD
:1045500092043097F1F0808191814097D1F40280EC
:10456000F381E02DF0939004E0938F040190F081AB
:10457000E02D80818770813019F40E94222202C0D0
:104580000E94B321E0918F04F091900487898D7F80
:10459000878B0F90CF91DF91089580E060E070E00D
:1045A0000E948A220895FF920F931F93CF93DF9367
:1045B0008C01F62EEA0122E8621711F40E94CD2246
:1045C000F80180819181009729F08558924009F087
:1045D0004FC049C080E060E070E040E050E020E083
:1045E00030E00E94031AF999FECF89E090E092BD75
:1045F00081BDF89A20B5F999FECF8AE090E092BD8E
:1046000081BDF89A90B5822F8B50803110F490952F
:10461000291328E1822F0E944B1981E00E94341651
:1046200088E00E94E1170E94743F8EE590E290932B
:104630008A048093890483ED90E2909386048093AA
:10464000850481E894E00E94DE268CE093E10E94DC
:10465000834086E10E94E11785E892E0F8019183AA
:10466000808381E009C08F2DBE010E948A22F4CF91
:10467000F8011182108283E0DF91CF911F910F9199
:10468000FF9008958091D7048F5F8093D704815065
:1046900008951F93CF93DF93EC01162F888580FF39
:1046A0001CC0EC81FD813097C1F0D093CE04C09343
:1046B000CD0482E08887CE0106960995992787FD6B
:1046C00090950297029710F0133829F4CE01BE019D
:1046D0000E94712302C081E08887DF91CF911F91F2
:1046E0000895CF92DF92EF92FF920F931F93CF9393
:1046F000DF938C017B01C090CD04D090CE04DC010F
:1047000018968C911897882341F118961C92C091A5
:10471000CB04D091CC040BC00C171D0729F0CE019F
:1047200067E8A8010E9449230990D881C02D2097ED
:1047300099F7D8011496ED91FC911597309769F08F
:104740000E151F0551F01093CE040093CD04C8013F
:10475000069663E840E050E00995E091CB04F091C3
:10476000CC040E171F07A1F4F8018081918190936A
:10477000CC048093CB040EC0808191818017910777
:1047800031F4D8018D919C919183808303C0FC0109
:10479000309791F7D092CE04C092CD04DF91CF91A3
:1047A0001F910F91FF90EF90DF90CF90089560914F
:1047B000CD047091CE040E94712308958AE88093FD
:1047C000D7041092D9041092D8041092CC041092FD
:1047D000CB041092CE041092CD0408951F93CF9372
:1047E000DF9380917A058823C1F010927A05C091F9
:1047F000CB04D091CC0411E00EC08985882341F010
:1048000018871986CE0162E840E050E00E944923F3
:104810000990D881C02D209781F72091D8042223B8
:1048200009F470C08091D90490E0FC01EE0FFF1FE5
:10483000EE0FFF1FE80FF91FE652FB4F60816093F8
:10484000D604418152815093D5044093D40403800F
:10485000F481E02DF093D304E093D20401968F719C
:1048600090708093D90421502093D804309709F098
:1048700042C08091CB049091CC049093D10480935A
:10488000D00411E031C080917A058823B9F01092EC
:104890007A05C091CB04D091CC040EC089858823C1
:1048A00041F018871986CE0162E840E050E00E948E
:1048B00049230990D881C02D209781F74091D404D5
:1048C0005091D5048091D0049091D1046091D60488
:1048D0000E944923E091D004F091D104808191811C
:1048E0009093D1048093D0048091D0049091D1040E
:1048F000892B49F607C0613811F481E08087CF0128
:104900000E94492380917A052091D80430E0280F35
:10491000311DC901DF91CF911F91089580917A05D2
:104920002091D80430E0280F311DC9010895DC0121
:104930002091D804203219F421E030E01AC080918F
:10494000D904820F8F718093CF0490E0FC01EE0FA9
:10495000FF1FEE0FFF1FE80FF91FE652FB4F6083AA
:1049600052834183B483A3832F5F2093D80420E034
:1049700030E0C90108950F931F930091CD04109169
:10498000CE040E9449231093CE040093CD041F91BE
:104990000F910895CF93DF93DC01EB016091CB047D
:1049A0004091CC04862F942F9C01F90103C0019003
:1049B000F081E02DEA17FB07B9F03097C1F76C934F
:1049C00011964C931197B093CC04A093CB0481E043
:1049D00018968C93189717961C921E921697CD01D5
:1049E00061E8AE010E94BB24DF91CF910895FC01E4
:1049F000009741F080858150823020F481E08187EA
:104A000080937A05089520E030E0FC0180858823BA
:104A100011F021E030E0C9010895CF93DF93C6E0A3
:104A2000D1E004C060E070E00E94CA2489919991AD
:104A30000097C1F7DF91CF910895FC0180819181AA
:104A400022813381820F931F918380830895EF9297
:104A5000FF920F931F93FC01E080F180028113818C
:104A60000E94E7140E0D1F1D081B190BC8011F9192
:104A70000F91FF90EF9008950F931F938C010E9468
:104A8000E71440E050E0F80120813181821B930B54
:104A9000228133818217930710F041E050E0CA0170
:104AA0001F910F9108950F931F938C010E94E7149B
:104AB000F801918380831F910F9108950F931F93A5
:104AC0008C01FC01738362830E94E714F8019183D7
:104AD00080831F910F91089520E030E0FC018681D2
:104AE0009781892B11F421E030E0C9010895FC0180
:104AF0002281338180819181280F391FC901089556
:104B0000FC0180819181089520917B0530917C0585
:104B10002115310511F021E030E0C901089580919F
:104B20007B0590917C05892B19F420E030E004C0CE
:104B300020917D0530917E05C901089580917B0506
:104B400090917C05892B29F410927E0510927D05A9
:104B500008950E94E714BC01E0917B05F0917C056B
:104B60004281538180819181480F591F461B570B09
:104B70000CC02281338180819181280F391F261B2F
:104B8000370B2417350708F4A9010480F581E02DBF
:104B9000309779F7460F571F50937E0540937D0558
:104BA0000895CF93DF93EC01E0917B05F0917C05B4
:104BB0008E179F0741F48C819D8190937C05809393
:104BC0007B0514C0FC01309731F0848195818C17EE
:104BD0009D07C1F707C01D821C821F821E82DF91C4
:104BE000CF9108958C819D81958384830E949E2519
:104BF000F2CFFC0180819181860F971F9183808382
:104C00000E949E25089582EB91E00E94F72408956A
:104C1000EF92FF920F931F93CF93DF937C01FC01E0
:104C200080819181009729F08A35910509F06DC046
:104C30000BC010927C0510927B058AE590E0F7018D
:104C40009183808381E065C0673849F59A01E091DE
:104C50007B05F0917C0503C00480F581E02D309741
:104C600041F38681978182179307B1F3E0937B0527
:104C7000F0937C050FC016968D919C911797821723
:104C8000930711F0FD0106C014968D919C91159724
:104C900095838483A481B581109769F7CECF62385C
:104CA00061F6C0917B05D0917C0500E010E02AC040
:104CB000CE010E943C25892B01F18E819F8168E8FD
:104CC000AE010E949724892BA1F41F821E828C8141
:104CD0009D810115110521F0F8019583848304C09D
:104CE00090937C0580937B051D821C820E949E25EB
:104CF000D8CF82EB91E00E94F7248E018C819D81B8
:104D00009C01E9012097A1F698CFF701118210824A
:104D100083E0DF91CF911F910F91FF90EF90089565
:104D2000CF93DF93EC0182EB91E00E94F7248E8118
:104D30009F81892B69F0E0917B05F0917C0506C08D
:104D4000EC17FD07A9F00480F581E02D3097C1F73D
:104D50008091CD049091CE049F838E8380917B05BA
:104D600090917C059D838C83D0937C05C0937B05BB
:104D70000E949E25DF91CF9108950F931F938C0180
:104D80000E945325C8010E9490261F910F910895FB
:104D90000F931F938C010E941D25C8010E9490262D
:104DA0001F910F9108950F931F938C010E945E2510
:104DB000C8010E9490261F910F910895FC019093C5
:104DC000800580937F050084F185E02D82E29CE2DE
:104DD000099584E197E20E94743091E09093A00AD3
:104DE0001092A10A8EEF8093A20A80E88093A30A12
:104DF0009093AA0A9093AB0A8AEA8093AC0A8093B4
:104E0000AD0A82E08093B80A0895BC0185E10E9452
:104E1000DB41E0917F05F0918005309721F004801F
:104E2000F581E02D09950895EF92FF920F931F935E
:104E3000DF93CF93CDB7DEB728970FB6F894DEBFD8
:104E40000FBECDBF8C0110928505109283050E9484
:104E500009420E9478419093820580938105809158
:104E6000E50C863029F483E062E070E00E94BC41EA
:104E70007E010894E11CF11C0115110521F4C70104
:104E800064E072E002C0C701B8010E941243E091E1
:104E90008105F09182053396F093B70AE093B60A44
:104EA000339780918305E80FF11D12821182809162
:104EB0008305E0918105F0918205E80FF11D83E003
:104EC00080838091E00C282F30E0C9018F709070B2
:104ED000892B09F03FC08091E10C9091E20C892B65
:104EE000C9F580918305E0918105F0918205E80F75
:104EF000F11D8181806481838091DF0C282F30E057
:104F0000C9018F709070892B81F48091E00C807FB3
:104F100061F480918305E0918105F0918205E80FAD
:104F2000F11D8181806881835FC0E091B60AF091B4
:104F3000B70A44E0220F331F4A95E1F78091E00C55
:104F400082958F70822B80838091B60A9091B70AE8
:104F5000019646C08091DF0C90E08F709070892B95
:104F600051F5822F807F39F580918305E09181058D
:104F7000F0918205E80FF11D818180688183E091C5
:104F8000B60AF091B70A9091E00C9F708091DF0C07
:104F9000807F982B9083E091B60AF091B70A8091B8
:104FA000E10C9091E20C928381838091B60A9091FA
:104FB000B70A039615C0E091B60AF091B70A80913E
:104FC000DF0C9091E00CA091E10CB091E20C808399
:104FD0009183A283B3838091B60A9091B70A049615
:104FE0009093B70A8093B60A8091E50C813161F401
:104FF00080918305E0918105F0918205E80FF11D14
:105000008181806281830EC0E091B60AF091B70A77
:1050100080838091B60A9091B70A01969093B70A5F
:105020008093B60A8091E60C803479F08F3FC9F006
:10503000813011F580918305E0918105F091820521
:10504000E80FF11D818188600AC080918305E0919D
:105050008105F0918205E80FF11D818180618183D6
:1050600019C080918305E0918105F0918205E80FD8
:10507000F11D81818861F3CFE091B60AF091B70A02
:1050800080838091B60A9091B70A01969093B70AEF
:105090008093B60A1092B80A31C0812F90E0FC01CB
:1050A00033E0EE0FFF1F3A95E1F7880F991FE80FE5
:1050B000F91FE056F54F80818130E9F4212F30E06F
:1050C000C90103E0880F991F0A95E1F7220F331FEA
:1050D000820F931F8E55954F67EE7CE048E050E0BD
:1050E0000E943F47009739F48AE0189FD0011124AD
:1050F000A056B54F09C01F5F1093B80A1091B80AA7
:10510000123058F2A0E0B0E0B093B50AA093B40A10
:10511000109709F49CC080918305E0918105F0917E
:105120008205E80FF11D11968C918295807F928106
:10513000892B828380918B0C92E089279091EF0CD0
:105140009817B1F59091F00C80918C0C981781F51F
:105150009091F10C80918D0C981751F59091F20C73
:1051600080918E0C981721F59091F30C80918F0C03
:105170009817F1F49091F40C8091900C9817C1F469
:105180009091F50C8091910C981791F49091F60CF8
:105190008091920C981761F480918305E0918105CC
:1051A000F0918205E80FF11D8281806C828365C0D9
:1051B0008091EF0C9091F00C892B59F58091F10CB6
:1051C0009091F20C892B29F58091F30C9091F40CBD
:1051D000892BF9F48091F50C87FD1BC08091830524
:1051E000E0918105F0918205E80FF11D82818068D0
:1051F0008283E091B60AF091B70A8091F50C909104
:10520000F60C918380838091B60A9091B70A02963A
:1052100030C080918305E0918105F0918205E80F0F
:10522000F11D8281806482832091B60A3091B70A91
:10523000C901DC01EFEEFCE088E001900D928150A5
:10524000E1F78091B60A9091B70A089612C0809152
:10525000B60A9091B70A9C01D901E7EEFCE080E123
:1052600001900D928150E1F78091B60A9091B70AB2
:1052700040969093B70A8093B60A8091F70C8F3FBF
:1052800009F065C08091F90C9091FA0C892B09F016
:1052900050C08091FB0C9091FC0C892B09F049C007
:1052A0008091FD0C9091FE0C892B09F042C08091F9
:1052B000FF0C9091000D892BE1F58091010D9091EB
:1052C000020D892BB1F58091030D9091040D892B6E
:1052D00081F58091050D882361F58091060D81503F
:1052E000823038F580918305E0918105F091820547
:1052F000E80FF11D828188608283E091B60AF09107
:10530000B70A80EA8083E091B60AF091B70A8091EB
:10531000F80C90E08F709070880F991F2081282BD7
:105320002083E091B60AF091B70A8091060D81833F
:10533000BFC08091B60A9091B70A9C01D901E7EFEE
:10534000FCE080E101900D928150E1F7E2C0109203
:10535000B80A31C0812F90E0FC0173E0EE0FFF1F0F
:105360007A95E1F7880F991FE80FF91FE056F54F7E
:1053700080818130E9F4212F30E0C90153E0880FAA
:10538000991F5A95E1F7220F331F820F931F8E55F5
:10539000954F67EF7CE048E050E00E943F47009760
:1053A00039F48AE0189FD0011124A056B54F09C0E6
:1053B0001F5F1093B80A1091B80A123058F2A0E09B
:1053C000B0E0B093B50AA093B40A109709F494C062
:1053D00080918305E0918105F0918205E80FF11D30
:1053E000828111969C91892B8283FE01319689815D
:1053F00092E089279091FF0C981779F59091000D14
:105400008181981751F59091010D8281981729F5A6
:105410009091020D8381981701F59091030D84817D
:105420009817D9F49091040D85819817B1F4909153
:10543000050D8681981789F49091060D878198173C
:1054400061F480918305E0918105F0918205E80F78
:10545000F11D82818C60828365C08091FF0C9091E8
:10546000000D892B59F58091010D9091020D892B2A
:1054700029F58091030D9091040D892BF9F4809109
:10548000050D87FD1BC080918305E0918105F0919A
:105490008205E80FF11D828188608283E091B60A5F
:1054A000F091B70A8091050D9091060D918380834C
:1054B0008091B60A9091B70A029630C08091830518
:1054C000E0918105F0918205E80FF11D82818460F1
:1054D00082832091B60A3091B70AC901DC01EFEF4F
:1054E000FCE088E001900D928150E1F78091B60ACE
:1054F0009091B70A089612C08091B60A9091B70AA7
:105500009C01D901E7EFFCE080E101900D92815010
:10551000E1F78091B60A9091B70A40969093B70A46
:105520008093B60A88E2809385058091E50C8131ED
:1055300009F064C09091070D8091080D805B904F39
:105540000F9770F59091090D80910A0D20EF803B27
:10555000920730F18F5B904F18F5E091B60AF09109
:10556000B70A8BEF8083E091B60AF091B70A909169
:105570000A0D905B8091080D8295807F980F918332
:10558000E091B60AF091B70A80910D0D90910E0D41
:10559000938382838091B60A9091B70A049625C0BE
:1055A000E091B60AF091B70A88EF8083E091B60ADD
:1055B000F091B70A8091070D9091080DA091090D07
:1055C000B0910A0D81839283A383B483E091B60ADC
:1055D000F091B70A80910D0D90910E0D9683858301
:1055E0008091B60A9091B70A07969093B70A809374
:1055F000B60A80918505885F80938505A091B60ADB
:1056000080918105A81BA093830580918505482F73
:1056100050E0E091890CF0918A0CE41BF50B2A2FE5
:1056200030E086E690E0821B930B7E010894E11C3B
:10563000F11C60918105709182058E179F0708F01B
:10564000D9C0CB0104964A2F50E00E945547E09103
:105650008105F09182058091890C90918A0C906C63
:105660009083E0918105F09182058091890C81837E
:10567000E0918105F09182058091990A8283E09101
:105680008105F09182058091980A8383809183053A
:105690008C5F8093830516E6412F481B487F40931B
:1056A00084056091810570918205680F711D2091BC
:1056B000850530E02152334FCB01B90150E00E9403
:1056C0004C47209183058091840590E0820F911DC5
:1056D0000E947341C7010E94052720918505809192
:1056E000840590E0820F911D9093970A8093960A0B
:1056F00085E080938305E0918105F091820580919A
:10570000890C90918A0C906E9083E0918105F091C4
:1057100082058091890C818380918305181B187FF5
:105720001093840587014CC0E0918105F0918205BA
:1057300083E0369527958A95E1F724836091890C5B
:1057400070918A0C4091960A5091970A9B01241BF4
:10575000350B8091840590E02817390720F4862FB7
:10576000841B8093840580918305609181057091ED
:105770008205680F711D409184052091960A309131
:10578000970A2152334FCB01B90150E00E944C4798
:10579000209183058091840590E0820F911D0E94E5
:1057A0007341C8010E940527209184058091960AC3
:1057B0009091970A820F911D9093970A8093960A71
:1057C0002091960A3091970A8091890C90918A0CC9
:1057D0002817390708F4A8CF8091980A9091990A60
:1057E00001969093990A8093980A1092970A1092C2
:1057F000960A1AC0260F371F4152534FC901BA01EA
:10580000AF010E944C47209183058091890C9091B3
:105810008A0C820F911D20918505821B91090E949F
:105820007341C7010E94052781E028960FB6F894BE
:10583000DEBF0FBECDBFCF91DF911F910F91FF90C3
:10584000EF9008951F93CF93DF93109285051092E8
:1058500083050E94784190938205809381058CE9AD
:105860009AE00E943C25892B41F01092950A1092F3
:10587000940A1092970A1092960AE0918105F0918D
:105880008205908180E02181422F50E0482B592BE6
:10589000CA018070987F892F9927803C910549F033
:1058A000803E9105A9F0C0E0D0E010E020E030E0BB
:1058B0001DC0EA01D770928180E0238130E0282B5F
:1058C000392B809183058C5F8093830510E00EC097
:1058D0001481928180E0238130E0282B392BEA016A
:1058E000D770809183058B5F809383058091960AA2
:1058F0009091970A892BF1F0209709F4E7C38091E2
:10590000940A9091950AC817D90709F0DFC38091CE
:105910009A0A90919B0A8217930709F0D7C384E1F2
:105920000E94D041BC0181E89CE00E942343892B66
:10593000C9F4CCC32097B1F0D093950AC093940AD0
:1059400030939B0A20939A0A8CE99AE067E771E00A
:105950000E945E2584E10E94D041BC0181E89CE068
:105960000E94124350918305553009F43DC32091A4
:10597000810530918205852F90E0D901A80FB91FCC
:105980004C91433021F0413409F0A0C315C3FC0110
:105990003396E20FF31FF093B70AE093B60A11961D
:1059A0008C9186FD22C087FD0DC081919191A191BE
:1059B000B1918093940590939505A0939605B0932B
:1059C00097050EC080E68093940580818F70809348
:1059D00095058181928190939705809396053396E2
:1059E000F093B70AE093B60A1BC087FD10C0808110
:1059F00082958F7080668093940581918295807FD7
:105A000080939505F093B70AE093B60A05C080E647
:105A10008093940510929505109297051092960523
:105A2000A0918105B091820580918305FD01E80F69
:105A3000F11D818185FD0BC0E091B60AF091B70A96
:105A4000819180939A05F093B70AE093B60A80910A
:105A50008305FD01E80FF11D818190E08871907050
:105A60008830910561F0893091051CF4892B79F01B
:105A700019C08031910529F04897A1F406C081E052
:105A800001C080E480939B050DC08FEFFBCFE091B8
:105A9000B60AF091B70A819180939B05F093B70AFB
:105AA000E093B60A80918305FD01E80FF11D828124
:105AB00090E08073907064E0959587956A95E1F722
:105AC000382F1092B80A20E02CC0822F90E0FC0101
:105AD00053E0EE0FFF1F5A95E1F7880F991FE80F6B
:105AE000F91FE056F54F80818130D1F4822F90E08C
:105AF000FC0173E0EE0FFF1F7A95E1F7880F991F05
:105B0000E80FF91FE056F54F8181831749F4209380
:105B1000B80A8AE0289FA00111244056554F07C0BB
:105B20002F5F223090F22093B80A40E050E050936B
:105B3000B50A4093B40A80918305A80FB11D12964F
:105B40008C91282F30E0207C30702034310509F40E
:105B500071C02134310524F4232B09F48BC0A0C07B
:105B600020383105D1F0203C310509F099C04115AC
:105B7000510509F439C2ACE9B5E0FA01329688E082
:105B800001900D928150E1F784E10E94D041BC0167
:105B90008CE995E00E94D63083C0A091B60AB091FE
:105BA000B70A8C9187FD23C04115510509F41CC229
:105BB000ACE9B5E0FA01329688E001900D9281508F
:105BC000E1F786E0E4EAF5E0DF011D928A95E9F766
:105BD000E091B60AF091B70A819191919093AB054B
:105BE0008093AA05F093B70AE093B60A59C080FDE6
:105BF000FBC111968C9111978150823008F0F4C14D
:105C00008FEF80939C058C9186958F7080939D0576
:105C10008DE02EE935E0F90111928A95E9F71196A8
:105C20008C9111978093AB051296B093B70AA0930D
:105C3000B60A36C04115510509F4D6C1ACE9B5E044
:105C4000FA01329688E001900D928150E1F7A4EAC2
:105C5000B5E08091B60A9091B70A9C01F90188E0FD
:105C600001900D928150E1F78091B60A9091B70AA8
:105C7000089612C0ACE9B5E08091B60A9091B70AD7
:105C80009C01F90180E101900D928150E1F7809132
:105C9000B60A9091B70A40969093B70A8093B60AD5
:105CA000A0918105B091820580918305FD01E80FE7
:105CB000F11D328133701092B80A20E02CC0822F7F
:105CC00090E0FC0153E0EE0FFF1F5A95E1F7880FBB
:105CD000991FE80FF91FE056F54F80818130D1F40C
:105CE000822F90E0FC0173E0EE0FFF1F7A95E1F741
:105CF000880F991FE80FF91FE056F54F8181831730
:105D000049F42093B80A8AE0289FA0011124405644
:105D1000554F07C02F5F223090F22093B80A40E021
:105D200050E05093B50A4093B40A80918305A80FC0
:105D3000B11D12968C91282F30E02C7030702430D9
:105D4000310509F471C02530310524F4232B09F401
:105D50008BC0A0C028303105D1F02C30310509F0BE
:105D600099C04115510509F43FC1ACEAB5E0FA010B
:105D7000329688E001900D928150E1F785E10E9412
:105D8000D041BC018CEA95E00E94D63083C0A0913E
:105D9000B60AB091B70A8C9187FD23C04115510511
:105DA00009F422C1ACEAB5E0FA01329688E001902C
:105DB0000D928150E1F786E0E4EBF5E0DF011D9202
:105DC0008A95E9F7E091B60AF091B70A819191912D
:105DD0009093BB058093BA05F093B70AE093B60A97
:105DE00059C080FD01C111968C911197815082306C
:105DF00008F0FAC08FEF8093AC058C9186958F7078
:105E00008093AD058DE02EEA35E0F90111928A9577
:105E1000E9F711968C9111978093BB051296B09378
:105E2000B70AA093B60A36C04115510509F4DCC083
:105E3000ACEAB5E0FA01329688E001900D9281500B
:105E4000E1F7A4EBB5E08091B60A9091B70A9C0106
:105E5000F90188E001900D928150E1F78091B60A36
:105E60009091B70A089612C0ACEAB5E08091B60AE4
:105E70009091B70A9C01F90180E101900D92815047
:105E8000E1F78091B60A9091B70A40969093B70ACD
:105E90008093B60A80918505885D80938505809101
:105EA0008305E0918105F0918205E80FF11D818164
:105EB00085FF56C0A091B60AB091B70A8C918C7F2D
:105EC000883F09F04DC081E180939A058C91883F0D
:105ED00029F18B3F09F088C0E4E9F5E0B896119606
:105EE0008C91119782958F7090E080559F40909390
:105EF000BC05818311968C91119790E08F70907002
:105F000080559F409283838312968D919C91139725
:105F10009093C3058093C205149619C011968D9174
:105F20009C9112979093BD058093BC0513968D911B
:105F30009C9114979093BF058093BE0515968D9103
:105F40009C9116979093C3058093C2051796B093C2
:105F5000B70AA093B60A80918505885F809385056E
:105F60008091B60A90918105891B809383052097C3
:105F700071F4109298050E94A6419091850598525F
:105F800020918305921B980F9093990508C0A897BC
:105F9000D0939805A8969E01285220939905809148
:105FA0009A05813109F58091980590919905909312
:105FB000C1058093C00518C0852F8F5F809383052E
:105FC000A4E9B5E0F901E80FF11D88E201900D9216
:105FD0008150E1F780918305885D809383058091EE
:105FE0008505885D809385050E94A6419091830573
:105FF000482F491B4093840580918505212F30E06F
:1060000053E0220F331F5A95E1F7280F311D2C560C
:106010003A4FE0918105F0918205E90FF11DC90128
:10602000BF0150E00E944C47CD2BC9F08091960AE9
:106030009091970A892B31F4809185058093960A77
:106040001092970A209184058091960A9091970A60
:10605000820F911D9093970A8093960A0BC020910E
:1060600085058091840590E0820F911D9093950A9B
:106070008093940A2091960A3091970A2115310550
:1060800039F08091940A9091950A28173907F1F414
:106090002FED3CE0E4E9F5E04091940A5091950A37
:1060A000C901BF010E944C478091940A9091950AC2
:1060B00090938A0C8093890C1092950A1092940AFE
:1060C0001092970A1092960A0E943635DF91CF916E
:1060D0001F910895E091B90AF091BA0A309711F42E
:1060E00080E00895099508959093BA0A8093B90ABB
:1060F0000895282F892F922F08959091E30C80E026
:106100002091E40CBC01620F711DAB01465C5F4F36
:10611000E7EEFCE0308120E08181D901A80FB11DBC
:106120004A0F5B1F4A175B0710F44F5F5F4F3296B1
:10613000BDE0E630FB0770F38DE0E630F80749F488
:10614000908180E0480F591F4817590710F44F5F9E
:106150005F4F6A5F724FE7E0FDE00EC0308120E0E4
:106160008181D901A80FB11D4A0F5B1F4A175B0738
:1061700010F44F5F5F4F3296E617F70778F3E61794
:10618000F70751F4908180E0480F591F48175907CD
:1061900018F44F5F5F4F06C04115510519F42FEFFA
:1061A0003FEF02C0342F252FC9010895CF93DF930D
:1061B000DC01EC012896FB0188E0019009928150F6
:1061C000E1F718968C91189792E0892718968C938E
:1061D000DF91CF910895539A5298E0E064E670E021
:1061E000F2E08BB1AB01417050709A01A3E0220F35
:1061F000331FAA95E1F7877F822B8BB98F2F8A9562
:10620000F1F789B190E084709070440F551F440FEE
:10621000551F8417950709F4EF5F6150704066239E
:1062200001F780E0E73408F081E008958AB1806AE0
:106230008AB98DB1806C8DB95F985D9A8EB1806C92
:106240008EB90E94EB30882319F081E08093BB0A5D
:106250000895BF92CF92DF92EF92FF920F931F9318
:10626000F0900013E0900113D0900213C09005133A
:10627000B090061310910713187F126020E030E0F1
:1062800040E050E060E07C2D8B2D912F00E10E94DA
:106290004D432F2920933C013E2930933D014D2948
:1062A00040933E0150933F01609340017093410140
:1062B00080934201909343018EEF809303138FEFFD
:1062C0008093041310930713E0912013F09121138E
:1062D0002F2D3E2D4D2D5EEF6FEF7C2D8B2D912FB1
:1062E00009951F910F91FF90EF90DF90CF90BF9095
:1062F0000895DC01FB018C91808311968C9111979C
:10630000818312968C91129782838FEF83838EEF15
:10631000848313968C911397858314968C9114978C
:10632000868315968C91878381E00895DC01FB01BB
:1063300080818C93818111968C9311978281129622
:106340008C931297858113968C931397868114965C
:106350008C931497878115968C9381E00895CF9341
:10636000DF93EC016623C1F041155105A9F020E04F
:1063700061501416150624F4FE01E60FF11D03C04A
:10638000FE01E20FF11DDF01A40FB51F80818C9388
:10639000662311F02F5FECCFDF91CF910895DC01E0
:1063A0000AC041508D91FB01E40FF11D90818917C6
:1063B00011F081E008954423A1F780E00895EF9261
:1063C000FF920F931F93CF93DF930E946C209093C3
:1063D000D5128093D4120E949115F82EE92E0E94B6
:1063E0009415482F02E512E1C8016F2D7E2D50E073
:1063F0000E944C470E949415F82EE8012E978AE9D6
:1064000090E80E9479309D878C87A091D412B0913A
:10641000D512ED91FC9111978181869586958370B7
:106420008230D1F41696ED91FC911797808191817D
:106430008F5F9F4F89F483E3809344128983809117
:10644000030D8A838091040D8B838091050D8C83CD
:106450008091060D8D8316C085E10E94D041FC011C
:106460008081809344128181809345128281809340
:1064700046128581809347128681809348128781D6
:106480008093491284E10E94D041FC018081809375
:106490004A12818180934B12828180934C128581B4
:1064A00080934D12868180934E12878180934F1284
:1064B0008EE0F80E84E492E16F2D70E041E00E94DE
:1064C000460780916B0C90916C0CA0916D0CB09173
:1064D0006E0C0196A11DB11D80936B0C90936C0CFA
:1064E000A0936D0CB0936E0CDF91CF911F910F9123
:1064F000FF90EF9008959C018091D61283FF03C016
:10650000C9010E94DF310895CF93DF93EC018091A0
:10651000D61283FF03C0CE010E94DF318091D612D4
:1065200080FF06C0E091D212F091D312CE010995FE
:10653000DF91CF910895BF92CF92DF92EF92FF92B9
:106540000F931F93DF93CF93CDB7DEB728970FB686
:10655000F894DEBF0FBECDBF7C016B018091D612D7
:1065600083FFA9C002E512E1FB01428160817181D4
:10657000C80150E00E944C47F601B28082EFC82E5D
:106580008FEFD82EC00ED11E8AE990E80E94793094
:10659000F60195878487F7018181869586958370BA
:1065A0008230B9F4858196818F5F9F4F91F483E3A8
:1065B00080934412F60181838091030D8283809140
:1065C000040D83838091050D84838091060D85835E
:1065D0002BC0F7018581898386818A8387818B839C
:1065E00080858C8381858D8382858E8383858F834F
:1065F000848588878E010F5F1F4FC80168E00E9465
:106600007420898180934412F8018181809345121E
:106610008281809346128581809347128681809380
:106620004812878180934912F70187858983808981
:106630008A8381898B8382898C8383898D838489F2
:106640008E8385898F83868988878E010F5F1F4F90
:10665000C80168E00E947420898180934A12F80181
:10666000818180934B12828180934C12858180932B
:106670004D12868180934E12878180934F12FEE0E7
:10668000BF0E84E492E16B2D70E040E00E9446076B
:1066900080916B0C90916C0CA0916D0CB0916E0C74
:1066A0000196A11DB11D80936B0C90936C0CA0936F
:1066B0006D0CB0936E0C28960FB6F894DEBF0FBE2B
:1066C000CDBFCF91DF911F910F91FF90EF90DF90A1
:1066D000CF90BF900895AC01DC01E2EEF1E086E0DE
:1066E00001900D928150E1F7CA0166E00E9474208A
:1066F00081E008952F923F924F925F926F927F9226
:106700008F929F92AF92BF92CF92DF92EF92FF92C1
:106710000F931F93DF93CF93CDB7DEB760970FB67C
:10672000F894DEBF0FBECDBF2C019FED692E9CE01B
:10673000792E6091E40C2091E30C88E2282E312C14
:10674000260C371C8091070D8538A1F0863848F457
:10675000813070F0853008F4E3C08058823040F416
:10676000DFC0893818F4873888F408C0893851F0B8
:106770008FEFD7C008E0A02EB12C0BC010E1A12EE6
:10678000B12C07C0B8E2AB2EB12C03C0A8E1AA2EF1
:10679000B12C922F80E0062F10E0082B192B0A193C
:1067A0001B090830110514F48EEFBBC0F7E0EF2E83
:1067B000FDE0FF2EEA0CFB1CD7018C918150119655
:1067C0009C91823008F092C0292F30E0E3E0220F44
:1067D000331FEA95E1F72250304090E00CC0E1E031
:1067E000F0E0EC0FFD1FEA0FFB1FAE0DBF1D129670
:1067F0008C9180839F5FA92FB0E0A217B3077CF331
:106800004114510421F5602F6650C701089648E0F5
:1068100050E00E94AF31F70132968981D70112967C
:106820008C938A8181838B818283BFEFB3838EEFC8
:1068300084838C8185838D8186838E818783E2E04A
:10684000D7011196EC9378E0C72ED12C1AC0F1E055
:106850004F16510411F08DEF64C0602F6E50C701C8
:10686000409648EF5FEF0E94AF31C70102960E9449
:106870006B33E1E0D7011196EC9368EFC62E6FEF12
:10688000D62E9090E30C88248091E40C90E0882927
:1068900099298C0D9D1DD30115968C9315971496EF
:1068A0009C938091890C90918A0C8C0D9D1D9093E6
:1068B0008A0C8093890CF101138212820E947D3030
:1068C00080959095D10113969C938E931297F70122
:1068D000818190E053E0880F991F5A95E1F7081BDA
:1068E000190B0C0D1D1DA80EB91E16C0292F30E066
:1068F000992319F400E010E008C0C90143E0880FB3
:10690000991F4A95E1F7081B190B93E0220F331FDB
:106910009A95E1F7A20EB31E083011050CF046CF90
:1069200080E060960FB6F894DEBF0FBECDBFCF916A
:10693000DF911F910F91FF90EF90DF90CF90BF906C
:10694000AF909F908F907F906F905F904F903F900F
:106950002F9008959C018091E50C8A3311F080E01E
:106960000895C9010E947A3308950E946C20909383
:10697000D5128093D4128DED96E80E9479309093D1
:10698000DE0C8093DD0CA091D412B091D512ED9164
:10699000FC91119781818695869583708230E9F408
:1069A0001696ED91FC911797808191818F5F9F4F93
:1069B000A1F483E38093D10C8093D20C8091030DDA
:1069C0008093D30C8091040D8093D40C8091050D9D
:1069D0008093D50C8091060D14C085E10E94D041B2
:1069E000FC0180818093D10C81818093D20C8281C3
:1069F0008093D30C85818093D40C86818093D50CB1
:106A000087818093D60C87ED9CE00E946B33809148
:106A1000D61282FF04C081E090E00E94AA34609107
:106A2000890C70918A0C625F7F4F70938A0C60931F
:106A3000890C81ED9CE041E00E94460780916B0C3F
:106A400090916C0CA0916D0CB0916E0C0196A11DF3
:106A5000B11D80936B0C90936C0CA0936D0CB09354
:106A60006E0C10928A0C1092890C08950E94B53415
:106A700008950F931F93DF93CF93CDB7DEB7289779
:106A80000FB6F894DEBF0FBECDBFDC011C968D9112
:106A90009C911D9786589D4D29F08CEB91E00E94AA
:106AA000B14728C08091D61281FF77C08C91833383
:106AB00031F411968C911197833381F541C08F3F4A
:106AC00069F511968C9111978F3F41F512968C9133
:106AD00012978F3F19F513968C9113978F3FF1F40E
:106AE00014968C9114978F3FC9F415968C91159735
:106AF0008F3FA1F480916F0C9091700CA091710C5C
:106B0000B091720C0196A11DB11D80936F0C9093F2
:106B1000700CA093710CB093720C3FC022EE31E068
:106B200046E04150BD01640F711DF9019081FB01E8
:106B30008081981791F52F5F3F4F442391F73CC018
:106B400000E010E08091890C90918A0C0E97909350
:106B50008A0C8093890C8091D61282FF04C080E059
:106B600090E00E94AA348091D61281FF16C0C8011D
:106B70000E946A308091670C9091680CA091690C1A
:106B8000B0916A0C0196A11DB11D8093670C909382
:106B9000680CA093690CB0936A0C10928A0C109246
:106BA000890C28960FB6F894DEBF0FBECDBFCF91EB
:106BB000DF911F910F9108958091FF0C92E089273A
:106BC00089838091000D8A838091010D8B83809150
:106BD000020D8C838091030D8D838091040D8E8333
:106BE0008091050D8F838091060D88878E010F5F40
:106BF0001F4FA8CF8091D6128F608093D6128091BC
:106C00007F0C9091800C9093D3128093D2120E94AB
:106C10007120FC019093E2118093E1110084F185D1
:106C2000E02D84E892E309958BE792E3909380044A
:106C300080937F0408951092DE121092DF1208955F
:106C40008AEE91E09093A1138093A0130895809110
:106C5000E80090E025E0969587952A95E1F7817008
:106C600008959C0195E09093E9008091E80085FDEE
:106C70000EC02FEF3FEF09C09093E9008091E8002C
:106C80008F778093E8001092DE12C9010895209357
:106C9000F1008091DE128F5F8093DE128091E80018
:106CA00085FFEACFF2CF8091DF128823C9F486E016
:106CB0008093E9008091E80082FF12C08091F30088
:106CC0008091F2008093DF12882351F48091E800D4
:106CD0008B7F8093E8008091E8008F778093E800B5
:106CE0008091DF12811181E008951F9386E08093E7
:106CF000E9008091DF12882319F40E945336FBCFFC
:106D00001091F1008091DF1281508093DF1288236F
:106D100051F48091E8008B7F8093E8008091E80037
:106D20008F778093E800812F90E00E943136812F89
:106D30001F91089585E08093E900E8EEF0E08081FE
:106D40008F7780831092DE1208951F93182F82E0B0
:106D50008093E9008091E80085FD04C080E090E028
:106D60001F9108950E945C04812F992787FD9095BB
:106D70000E943136F3CF80914601909147010097F0
:106D800019F422E037E007C0019719F027E537E052
:106D900002C023E636E0C901089582E1089580919A
:106DA000460190914701009719F424E137E007C0AC
:106DB000019719F029E637E002C025E736E0C9015E
:106DC00008958091460190914701009711F483E462
:106DD0000895019711F080E208958DE8089590914B
:106DE000EB0091609093EB008093EC008091ED00BC
:106DF0008270862B8093ED008091ED0082608093FD
:106E0000ED008091EE00881F8827881F08959091DB
:106E1000F40080E090FD06C08F5F873011F09695FA
:106E2000F9CF80E00895FB018093E90004C08191CF
:106E30008093F10041508091E80085FF02C0442317
:106E4000B1F7842F0895FB018093E90004C080917D
:106E5000F100819341508091E80085FF02C04423F6
:106E6000B1F7842F08958093E900EBEEF0E0808184
:106E70008062808308958091D8008F7B8093D800B2
:106E80008091D90081FF21C01092E9008091EB0030
:106E900080FD1BC01092E9008091EB00816080931F
:106EA000EB0082E08093EC008091ED0082708063C3
:106EB0008093ED008091ED0082608093ED008091E1
:106EC000EE00881F8827881F089580E0089583308A
:106ED00031F5613069F0613028F0623079F063306B
:106EE000F1F412C084E080937A0C83EC97E011C037
:106EF0008CE080937A0C89E897E00BC082E2809363
:106F00007A0C85E997E005C08CE080937A0C87EBDA
:106F100097E090937C0C80937B0C81E0089580E057
:106F200008958091E800877F8093E8008091D712D0
:106F30008093F1008091D8128093F1008091D91252
:106F40008093F1008091DA128093F1008091DB123E
:106F50008093F1008091DC128093F1008091DD122A
:106F60008093F1008091E8008E7F8093E80080910B
:106F7000E80080FFFCCF8091E80082FFFCCF809189
:106F8000E8008B7F8093E8008091E8008F77809302
:106F9000E80008958091E800877F8093E800809161
:106FA000E80082FFFCCF8091F1008093D71280919E
:106FB000F1008093D8128091F1008093D9128091D2
:106FC000F1008093DA128091F1008093DB128091BE
:106FD000F1008093DC128091F1008093DD128091AA
:106FE000E8008B7F8093E8008091E8008F778093A2
:106FF000E8008091E8008E7F8093E8008091E800AF
:1070000080FFFCCF08958091E800877F8093E8009F
:107010008091E8008E7F8093E8008091E80080FFF7
:10702000FCCF089580914601909147010297A8F402
:1070300081E08093E90081EC60E30E94EF3682E01A
:107040008093E90081E864E30E94EF3683E0809357
:10705000E90080E864E30E94EF3680914601909158
:1070600047010197A9F484E08093E90081EC60E294
:107070000E94EF3685E08093E90081E864E20E9497
:10708000EF3686E08093E90080E864E20E94EF3604
:107090008091460190914701029771F481E08093BD
:1070A000E90081E860E30E94EF3682E08093E90026
:1070B00080E860E30E94EF3620914601309147015D
:1070C0002230310510F582E08093EA001092EA0048
:1070D00084E08093EA001092EA0088E08093EA005E
:1070E0001092EA002130310581F480E18093EA00BA
:1070F0001092EA0080E28093EA001092EA0080E4B5
:107100008093EA001092EA0008952230310551F48C
:1071100080E28093EA001092EA0080E48093EA0023
:107120001092EA000895DF93CF9300D0CDB7DEB779
:107130008091F1008091F100613209F44CC062321B
:1071400038F46130E9F0613060F0603241F446C0FB
:107150006E3F71F16F3F08F5623209F442C080E082
:107160004FC08091F1008091F1008091F1008983FE
:107170008091F1008A8389819A810E946F0E40C0BC
:107180008091F1008091F1008091F10089838091DC
:10719000F1008A830E94420933C08091E800877F12
:1071A0008093E8008091E8008E7F8093E80027C0FC
:1071B0008091E800877F8093E8000E946D3D8150B8
:1071C0008093F1008091E8008E7F8093E80081E059
:1071D0008093E01215C00E94913711C00E94CA37F7
:1071E0000EC08091E800877F8093E8008091E800DE
:1071F0008E7F8093E8008091E80080FFFCCF81E0E3
:107200000F900F90CF91DF910895DF93CF93CDB77B
:10721000DEB762970FB6F894DEBF0FBECDBF4091C8
:10722000E91280E789831A828091F6128B831C828F
:107230001D821E821F828AE0888719861A861B8615
:107240001C868091F7128D878091F8128E871F8699
:10725000188A198A1A8A9E012F5F3F4FF90103C0CD
:1072600081918093F1008E2F821B8417C8F3809147
:10727000E8008F778093E8008091E1129091E2120C
:10728000A091E312B091E412841B9109A109B10904
:107290008093E1129093E212A093E312B093E41270
:1072A0001092F5121092F6121092F7121092F81234
:1072B00081E062960FB6F894DEBF0FBECDBFCF91CE
:1072C000DF9108958091E61290E083709070892B91
:1072D00009F05CC08091E712882309F057C06091E3
:1072E000E912613608F060E690E0E3EEF7E01EC0D8
:1072F000983019F4E7ECF7E009C0903119F4EFEC9D
:10730000F7E004C0903211F4EFEDF7E08491809340
:10731000F1009F5F943249F42091E1123091E21222
:107320004091E3125091E41214C03196961700F385
:10733000F3CF903459F48091E8008F778093E80080
:107340002054304040405040605490E01092F10092
:107350009F5F961770F38091E8008F778093E80025
:10736000261B3109410951092093E1123093E212A1
:107370004093E3125093E4121092F5121092F61219
:107380001092F7121092F81281E0089581E0809334
:10739000F51285E08093F61284E28093F712109242
:1073A000F81280E008951092F5121092F6121092E1
:1073B000F7121092F81281E008951092F5121092CF
:1073C000F6121092F7121092F812089581E080934D
:1073D000F51282E08093F6128AE38093F7121092FE
:1073E000F812089581E08093F51286E08093F612FA
:1073F00088E28093F7121092F812089581E080934A
:10740000F51284E08093F6121092F7121092F8129F
:10741000089581E08093F51287E08093F61287E269
:107420008093F7121092F81208951F93182F882353
:1074300011F01092F1006093F1001092F100809130
:107440007E0C0E949C3D882321F080E88093F1000F
:1074500002C01092F100112331F01092F10010924D
:10746000F1001092F1001092F1001F9108950F9316
:107470001F93182F882319F00091ED1202C000917C
:10748000E9128091E71290E08F7390708C31910532
:1074900041F08F33910509F458C0019709F0E5C018
:1074A00021C0812F6FE00E94153A8CE18093F1009A
:1074B0008AE08093F1001092F10085E08093F10062
:1074C0001092F1001092F1001092F1001092F10070
:1074D0001092F1001092F1001092F10081E080937F
:1074E000F10022C0812F6FE00E94153A81E0809365
:1074F000F1008AE08093F10090E89093F10083E03E
:107500008093F1001092F1001092F1001092F100BE
:107510001092F1000D3040F09093F1001092F100C4
:107520001092F1001092F1008091E8008F77809323
:10753000E8008091E1129091E212A091E312B091E3
:10754000E4124097A109B1092BC0812F6BE10E9481
:10755000153A112399F0083061F58091E8008F7792
:107560008093E8008091E1129091E212A091E312E1
:10757000B091E4120897A109B10912C00430C9F40E
:107580008091E8008F778093E8008091E1129091DC
:10759000E212A091E312B091E4120497A109B1099B
:1075A0008093E1129093E212A093E312B093E4125D
:1075B00069C071E07093F1006AE06093F10090E8B7
:1075C0009093F10083E08093F1001092F10010920B
:1075D000F1001092F1001092F1002091E11230912F
:1075E000E2124091E3125091E4120D3060F1909359
:1075F000F1001092F1001092F1001092F1008CE174
:107600008093F1006093F1001092F10085E0809387
:10761000F1001092F1001092F1001092F10010921E
:10762000F1001092F1001092F1001092F1007093AD
:10763000F1008091E8008F778093E8002C51304072
:107640004040504009C08091E8008F778093E80067
:10765000201B3109410951092093E1123093E212B4
:107660004093E3125093E4120DC081E08093F51231
:1076700085E08093F61284E28093F7121092F8125C
:1076800080E009C01092F5121092F6121092F712D3
:107690001092F81281E01F910F9108950F931F939C
:1076A000DF93CF9300D000D000D0CDB7DEB7FE017E
:1076B00033968091E71283838091E81282838091D0
:1076C000E91281838091EA128B838091EC128A8384
:1076D0008091ED12898309811A810115110509F440
:1076E00063C080917E0C0E949C3D813039F4809370
:1076F000F51287E08093F61287E23FC04B815C81F0
:107700006D817E8180917E0C98010E94713D823056
:10771000910561F183309105B1F1892BE1F510926A
:10772000F5121092F6121092F7121092F8129801B8
:1077300040E050E089E0220F331F441F551F8A9517
:10774000D1F78091E1129091E212A091E312B091F1
:10775000E412821B930BA40BB50B8093E112909360
:10776000E212A093E312B093E41226C081E080936A
:10777000F51282E08093F6128AE38093F71210925A
:10778000F81280E01AC081E08093F51286E08093C1
:10779000F61288E2F2CF81E08093F51284E08093C4
:1077A000F6121092F712EBCF1092F5121092F61219
:1077B0001092F7121092F81281E026960FB6F89404
:1077C000DEBF0FBECDBFCF91DF911F910F91089506
:1077D0000F931F93DF93CF9300D000D000D0CDB78D
:1077E000DEB7FE0133968091E71283838091E81221
:1077F00082838091E91281838091EA128B83809148
:10780000EC128A838091ED12898309811A81011516
:10781000110509F456C04B815C816D817E81809198
:107820007E0C98010E94833D8230910561F1833086
:10783000910589F1892BC9F51092F5121092F61273
:107840001092F7121092F812980140E050E099E07F
:10785000220F331F441F551F9A95D1F78091E112D3
:107860009091E212A091E312B091E412821B930B6B
:10787000A40BB50B8093E1129093E212A093E31254
:10788000B093E41226C081E08093F51282E08093E9
:10789000F6128AE307C081E08093F51286E08093B8
:1078A000F61288E28093F71208C081E08093F51207
:1078B00084E08093F6121092F7121092F81280E092
:1078C00009C01092F5121092F6121092F71210924F
:1078D000F81281E026960FB6F894DEBF0FBECDBF3A
:1078E000CF91DF911F910F9108950F931F93DF9315
:1078F000CF9300D000D0CDB7DEB780917E0C8E0143
:107900000F5F1F4FB8010E94A33D8230910509F41B
:107910003FC08330910509F443C0892B09F04AC068
:10792000F80183818093F10082818093F10081814D
:107930008093F10080818093F1001092F100109209
:10794000F10082E08093F1001092F1008091E80054
:107950008F778093E8008091E1129091E212A091DC
:10796000E312B091E4120897A109B1098093E112E2
:107970009093E212A093E312B093E4121092F512E6
:107980001092F6121092F7121092F81281E01DC0B8
:1079900081E08093F51282E08093F6128AE307C0BB
:1079A00081E08093F51286E08093F61288E280935E
:1079B000F71208C081E08093F51284E08093F612FC
:1079C0001092F7121092F81280E00F900F900F9023
:1079D0000F90CF91DF911F910F91089580917E0CB0
:1079E0000E94AE3D8230910551F08330910579F0CF
:1079F000892BB9F41092F5121092F61218C081E09A
:107A00008093F51282E08093F6128AE307C081E04A
:107A10008093F51286E08093F61288E28093F71245
:107A200008C081E08093F51284E08093F6121092F2
:107A3000F7121092F81281E008958091E5128A32CF
:107A400029F477980E944E3B779A0895883229F45A
:107A50005D980E94E83B5D9A08958A3109F18B3167
:107A600038F4833089F0823191F0882399F028C06E
:107A7000853299F0863218F48E3111F513C08F32A9
:107A800089F08A35E9F418C00E94053908950E94EA
:107A9000623908950E94EE3C08950E94753C089555
:107AA00080E00BC01092F5121092F6121092F712AD
:107AB0001092F81281E0089581E00E94373A08950B
:107AC00081E08093F51285E08093F61280E2809346
:107AD000F7121092F81280E0089581E0089580E096
:107AE0000895882319F020E030E00BC0CB01BA01E3
:107AF000A9010E94553F9C01009719F40E94713F13
:107B00009C01C9010895882319F020E030E00BC0E2
:107B1000CB01BA01A9010E94733E9C01009719F4A0
:107B20000E946E3F9C01C9010895882311F081E0F5
:107B300008950E94CE3D0895882311F081E00895B4
:107B40000E94CC3D0895882319F021E030E004C064
:107B5000CB010E94BC3D9C01C9010895882319F006
:107B600021E030E003C00E94B93D9C01C9010895A5
:107B7000089580E090E00895FC018091F8019091D3
:107B8000F901A091FA01B091FB0180839183A28356
:107B9000B38380E090E0089580E0089580E0089548
:107BA00060587F4F8F4F9F4F29E0660F771F881FC8
:107BB000991F2A95D1F76093F9127093FA12809366
:107BC000FB129093FC1281E0089508955F926F92EA
:107BD0007F928F929F92AF92BF92CF92DF92EF925D
:107BE000FF920F931F93CF93DF93BC01A090F912E4
:107BF000B090FA12C090FB12D090FC12EC0135014B
:107C00004601D401C301562D492F3A2F2B2FF8E0FE
:107C10005F2EF894852F942FA32FB22F9C01AD01D6
:107C2000E0E4EE2EF12C012D112DE20EF31E041FC7
:107C3000151F4BBFF90187918093F1002F5F3F4FD4
:107C40004F4F5F4F2E153F054007510791F7809129
:107C5000E8008F778093E80078948091E80085FFB2
:107C6000FCCF5A9439F0DA01C901522F492F3A2F2B
:107C70002B2FCFCF219780E092E0A0E0B0E0680EFC
:107C8000791E8A1E9B1E209709F0BBCFA80EB91E35
:107C9000CA1EDB1E61507040CB01A0E0B0E039E0AD
:107CA000880F991FAA1FBB1F3A95D1F7A80EB91EBE
:107CB000CA1EDB1EA092F912B092FA12C092FB12F9
:107CC000D092FC1281E0DF91CF911F910F91FF9034
:107CD000EF90DF90CF90BF90AF909F908F907F906C
:107CE0006F905F90089560587F4F8F4F9F4FA9E02E
:107CF000660F771F881F991FAA95D1F76093F91215
:107D00007093FA128093FB129093FC12CA010E94A6
:107D1000E63D80E090E0089560587F4F8F4F9F4F81
:107D2000B9E0660F771F881F991FBA95D1F7609346
:107D3000F9127093FA128093FB129093FC1281E077
:107D4000089508957F928F929F92AF92BF92CF92A3
:107D5000DF92EF92FF920F931F93CF93DF934C012B
:107D6000C0E0D0E0CC24DD2488E0782E86C080916D
:107D7000E80085FFFCCFF894209799F40091F91260
:107D80001091FA122091FB123091FC12E091000246
:107D9000F091010260E070E080E090E040E050E0AF
:107DA000099500E4A02EB12CAC0EBD1E9091F100FF
:107DB0008091F1004091F9125091FA126091FB12FA
:107DC0007091FC12F82EEE248701090F111DE0912D
:107DD000FC01F091FD0180E090E09E010995229662
:107DE000CA15DB0519F78091E8008B7F8093E800C6
:107DF0008091E8008F778093E80081E0C030D80759
:107E0000D9F50091F9121091FA122091FB123091DC
:107E1000FC12E091FE01F091FF0160E070E080E073
:107E200090E040E050E0099578948091F9129091AB
:107E3000FA12A091FB12B091FC1280509F4FAF4FED
:107E4000BF4F8093F9129093FA12A093FB12B09354
:107E5000FC1280E091E0C80ED91E90E0C91692E0B5
:107E6000D90619F0C0E0D0E007C008948108910855
:107E7000C0E0D0E0CC24DD247A94772009F077CFDD
:107E80008114910419F018E0712E71CF81E0DF9117
:107E9000CF911F910F91FF90EF90DF90CF90BF9007
:107EA000AF909F908F907F90089560587F4F8F4F35
:107EB0009F4F29E0660F771F881F991F2A95D1F7DA
:107EC0006093F9127093FA128093FB129093FC1254
:107ED000CA010E94A23E80E090E0089580E090E018
:107EE000089580E090E008959F92AF92BF92CF9264
:107EF000DF92EF92FF920F931F93DF93CF93CDB753
:107F0000DEB728970FB6F894DEBF0FBECDBF81E075
:107F10000E9487208CE260EF44E022E00E94E11B97
:107F20008DEC9BEA0E943C1710910013F090011316
:107F3000E0900213D0900313C0900413B090051387
:107F4000A0900613909007131983212F3F2D4E2DDB
:107F50005D2D6C2D7B2D8A2D992D08E00E944D43BF
:107F60002A83212F3F2D4E2D5D2D6C2D7B2D8A2DAB
:107F7000992D00E10E944D432B83212F3F2D4E2D43
:107F80005D2D6C2D7B2D8A2D992D08E10E944D438E
:107F90002C83212F3F2D4E2D5D2D6C2D7B2D8A2D79
:107FA000992D00E20E944D432D83212F3F2D4E2D10
:107FB0005D2D6C2D7B2D8A2D992D08E20E944D435D
:107FC0002E83212F3F2D4E2D5D2D6C2D7B2D8A2D47
:107FD000992D00E30E944D432F83212F3F2D4E2DDD
:107FE0005D2D6C2D7B2D8A2D992D08E30E944D432C
:107FF000288780E093E10E94E11682ED94E00E94E0
:10800000F0460E94EB468093FD12ABE8BCE0E0E056
:10801000F3E188E001900D928150E1F78BE89CE05C
:1080200068E00E94742028960FB6F894DEBF0FBE59
:10803000CDBFCF91DF911F910F91FF90EF90DF9017
:10804000CF90BF90AF909F9008959093FF12809330
:10805000FE1208958091FE129091FF120895809370
:108060004B13089580914B1308952093421330933E
:1080700043134093441350934513609346137093F6
:108080004713809348139093491308952091421306
:10809000309143134091441350914513609146131E
:1080A00070914713809148139091491308959093CC
:1080B0000B1380930A13089580910A1390910B1368
:1080C000089520933A1330933B1340933C135093FD
:1080D0003D1360933E1370933F138093401390932E
:1080E0004113089520913A1330913B1340913C1372
:1080F00050913D1360913E1370913F138091401356
:10810000909141130895FC018DE391E49183808364
:108110008AE391E49383828385E391E49583848366
:108120008FE291E49783868385E290E4918780874C
:108130008AE290E49387828788E291E49587848736
:1081400081E291E4978786878FE290E4918B808B20
:1081500082E390E4938B828B8CE091E4958B848B0B
:1081600087EF90E4978B868B80EF90E4918F808FE0
:1081700089EE90E4938F828F84EE90E4958F848FC4
:108180008DED90E4978F868F85E390E491A380A393
:1081900086E490E493A382A387E590E495A384A367
:1081A0008CE590E497A386A381E690E491A780A74D
:1081B00082E790E493A782A708950E94AD178111EA
:1081C00081E080934A13089580934A130E942D16EC
:1081D00008950E948B1780930813909309130895B4
:1081E00080930813909309130E943017089580E03C
:1081F00093E10E94481720910013309101134091A0
:108200000213509103136091041370910513809130
:1082100006139091071308952093001330930113D0
:108220004093021350930313609304137093051348
:10823000809306139093071380E093E10E94E11668
:1082400008950E949C1780933813909339130895D2
:1082500080933813909339130E943C1708950E941D
:10826000451980934C1390E0089580934C130E941D
:108270004B1908950E94CE1708950E94B9170895CA
:10828000AC012091C10A822F90E04817590734F4BD
:10829000241B2093C10A21E030E004C01092C10ADF
:1082A00020E030E0C90108954091BD0A5091BE0A16
:1082B0009C014817590718F420E030E012C0809163
:1082C000BF0A9091C00A820F931F9093C00A8093B7
:1082D000BF0A421B530B5093BE0A4093BD0A21E0D4
:1082E00030E0C90108959093BE0A8093BD0A0895B5
:1082F0008091BF0A9091C00AC096209102023091ED
:108300000302280F391FC90108958091C10A2091E5
:10831000020230910302280F311DC901089540E087
:1083200050E08091020290910302C0962091C20A0F
:108330003091C30A2817390711F041E050E0CA0113
:1083400008958091C20A9091C30A08958091BD0A50
:108350009091BE0A08959091C10A80E3891B089507
:1083600080E39091C10A891B2091BD0A3091BE0A19
:10837000280F311DC9010895E82FF0E0EE0FFF1F0F
:10838000E259FC4E7183608381E090E00895E82F0C
:10839000F0E0EE0FFF1FE259FC4E808191810895BD
:1083A000282F30E043E0220F331F4A95E1F7225592
:1083B0003D4EC901089590E053E0880F991F5A95EA
:1083C000E1F782559D4E0E94124381E090E00895AE
:1083D000EEE6F3E11192119283E1E639F807D1F765
:1083E0008EE493E164E072E00E94124386E593E13B
:1083F00064E072E00E9412438EE593E164E072E073
:108400000E94124386E693E164E072E00E94124308
:1084100008951092C00A1092BF0A1092BE0A1092DC
:10842000BD0A80E38093C10A809102029091030209
:10843000C0969093C30A8093C20A0E94E8410895AF
:10844000EF92FF920F931F938C017B010E940942D0
:108450001093C30A0093C20AF092BE0AE092BD0ACA
:108460001F910F91FF90EF900895AEE6B3E1FC01EC
:1084700088E201900D928150E1F7AEE4B3E1FB0197
:1084800080E201900D928150E1F70895DC01EEE663
:10849000F3E188E201900D928150E1F7DB01EEE417
:1084A000F3E180E201900D928150E1F70895EF929F
:1084B000FF920F931F937C018091C10A90E000E32B
:1084C00010E0F801E81BF90B209102023091030241
:1084D000280F391FC701B901AF010E944C47809195
:1084E000C10A081B11090E0D1F1D2091C20A3091EF
:1084F000C30A8091BF0A9091C00A280F391F40918A
:10850000BD0A5091BE0AC801B9010E944C47209192
:10851000BD0A3091BE0A205D3F4F8091C10A281BE1
:108520003109C9011F910F91FF90EF9008950F93AA
:108530001F934091C10A50E000E310E0F801E41BF2
:10854000F50B2091020230910302240F351FB9016F
:10855000AF010E944C478091C10A081B1109C80154
:108560001F910F910895E091C20AF091C30A6091A2
:108570000202709103029B01205D3F4FE217F30757
:1085800049F04091BD0A5091BE0AC901BF010E9445
:108590004C4708958091BF0A9091C00A0097D9F086
:1085A0004091BD0A5091BE0A405D5F4FDC01D096FC
:1085B000A60FB71F20E330E007C0FB01E20FF31F57
:1085C0008D9180832F5F3F4F24173507B4F31092AE
:1085D000C00A1092BF0A0895EF92FF920F931F9363
:1085E000F82EE92E162F072F0E940942212F302F37
:1085F000C9018C018138910510F000E810E08091EC
:10860000C20A9091C30A6F2D7E2DA8010E944C478B
:108610001093BE0A0093BD0AC8011F910F91FF90ED
:10862000EF900895AC0120E030E0FA01E20FF31F73
:10863000DB01A20FB31F8C9180832F5F3F4F283047
:10864000310599F70895AC0120E030E0FA01E20F1E
:10865000F31FDB01A20FB31F90818C91981719F0C3
:1086600020E030E007C02F5F3F4F2830310571F721
:1086700021E030E0C9010895AC0120E030E0F901CB
:10868000EA56FC4EDA01A20FB31F8C9180832F5F54
:108690003F4F2830310599F70895EF92FF920F93DD
:1086A000DF93CF93CDB7DEB760970FB6F894DEBFF8
:1086B0000FBECDBFA82F002309F461C07E0108942E
:1086C000E11CF11C88E0F70111928A95E9F72983F2
:1086D0003A834B835C836D837E83AF83988780E28C
:1086E000801BE82FFF27E7FDF0954D815E816F81AC
:1086F0007885181684F01D861E861F86188A88279E
:1087000099278E1B9F0B04C07695679557954795C3
:108710008A95D2F728C0202F332727FD3095DB011B
:10872000CA01022E04C0B695A795979587950A941D
:10873000D2F78D879E87AF87B88B04C0440F551F33
:10874000661F771FEA95D2F789819A81AB81BC8138
:1087500004C0B695A795979587952A95D2F7482B8B
:10876000592B6A2B7B2B49875A876B877C872985F6
:108770003A854B855C856D857E85AF8598898A2F86
:1087800060960FB6F894DEBF0FBECDBFCF91DF91DC
:108790000F91FF90EF900895A8E1B0E0E2EDF3E4CF
:1087A0000C94964A69837A838B839C832D833E83C2
:1087B0004F83588789E0E82EF12CEC0EFD1ECE0188
:1087C0000196B7010E94C9458E010F5E1F4FCE0171
:1087D0000596B8010E94C9458985823040F0898993
:1087E000823028F0C701B8010E94414601C08FEFD6
:1087F0006896E6E00C94B24AA8E1B0E0E2E0F4E466
:108800000C94964A69837A838B839C832D833E8361
:108810004F83588789E0E82EF12CEC0EFD1ECE0127
:108820000196B7010E94C9458E010F5E1F4FCE0110
:108830000596B8010E94C9458985823040F0898932
:10884000823028F0C701B8010E94414601C081E092
:108850006896E6E00C94B24AA8E0B0E0E2E3F4E403
:108860000C94924A7B018C0161157105810591057B
:1088700019F482E0898360C083E089838EE1C82E89
:10888000D12CDC82CB82ED82FE820F831887C80157
:10889000B7010E94A544FC013197F7FF3BC0222796
:1088A00033272E1B3F0B57016801022E04C0D694BC
:1088B000C794B794A7940A94D2F740E050E060E0E0
:1088C00070E081E090E0A0E0B0E004C0880F991F64
:1088D000AA1FBB1F2A95D2F70197A109B1098E21C2
:1088E0009F21A023B1230097A105B10521F041E00C
:1088F00050E060E070E04A295B296C297D294D83B6
:108900005E836F8378878EE190E08E1B9F0B9C8344
:108910008B8312C0309781F00E2E04C0EE0CFF1C2A
:10892000001F111F0A94D2F7ED82FE820F83188771
:10893000CE1ADF0ADC82CB821A82CE0101960E9417
:10894000F4442896EAE00C94AE4AEF92FF920F931B
:108950001F937B018C0180E0E81680E0F80681E03F
:10896000080780E0180788F48FEFE816F104010586
:10897000110531F028F088E090E0A0E0B0E017C0E9
:1089800080E090E0A0E0B0E012C080E0E81680E077
:10899000F80680E0080781E0180728F088E190E0F9
:1089A000A0E0B0E004C080E190E0A0E0B0E020E210
:1089B00030E040E050E0281B390B4A0B5B0B04C051
:1089C00016950795F794E7948A95D2F7F701E45F37
:1089D000FD4F8081281B310941095109C9011F91AF
:1089E0000F91FF90EF900895DF92EF92FF920F9317
:1089F0001F93FC01E480F58006811781D18080817E
:108A0000823048F480E090E0A0E1B0E0E82AF92A62
:108A10000A2B1B2BA5C0843009F49FC0823021F49F
:108A2000EE24FF24870105C0E114F10401051105BE
:108A300019F4E0E0F0E096C0628173819FEF623844
:108A400079070CF05BC022E83FEF261B370B2A3179
:108A500031052CF020E030E040E050E02AC0B801C1
:108A6000A701022E04C076956795579547950A94FD
:108A7000D2F781E090E0A0E0B0E004C0880F991F39
:108A8000AA1FBB1F2A95D2F70197A109B1098E2110
:108A90009F21A023B1230097A105B10521F081E01A
:108AA00090E0A0E0B0E09A01AB01282B392B4A2BD3
:108AB0005B2BDA01C9018F779070A070B0708034A1
:108AC0009105A105B10539F427FF09C0205C3F4F8E
:108AD0004F4F5F4F04C0215C3F4F4F4F5F4FE0E06F
:108AE000F0E02030A0E03A07A0E04A07A0E45A07EF
:108AF00010F0E1E0F0E079018A0127C060387105EB
:108B000064F5FB01E158FF4FD801C7018F779070E2
:108B1000A070B07080349105A105B10539F4E7FE6D
:108B20000DC080E490E0A0E0B0E004C08FE390E0EE
:108B3000A0E0B0E0E80EF91E0A1F1B1F17FF05C0DA
:108B400016950795F794E794319687E01695079563
:108B5000F794E7948A95D1F705C0EE24FF248701A6
:108B6000EFEFF0E06E2F679566276795902F9F7760
:108B7000D794DD24D7948E2F8695492F462B582FD6
:108B80005D29B701CA011F910F91FF90EF90DF900F
:108B90000895FC01DB01408151812281622F6F77B2
:108BA00070E0221F2227221F9381892F880F822B9A
:108BB000282F30E0991F9927991F11969C931197A0
:108BC00021153105A9F5411551056105710511F40E
:108BD00082E037C082E89FEF13969C938E931297A2
:108BE0009A01AB0167E0220F331F441F551F6A959E
:108BF000D1F783E08C930DC0220F331F441F551F04
:108C000012968D919C911397019713969C938E9336
:108C10001297203080E0380780E0480780E458074A
:108C200058F314962D933D934D935C9317970895A5
:108C30002F3F310579F4411551056105710519F48E
:108C400084E08C93089564FF03C081E08C9312C08C
:108C50001C9210C02F57304013963C932E931297BE
:108C600083E08C9387E0440F551F661F771F8A951A
:108C7000D1F7706414964D935D936D937C93179721
:108C800008951F93DC01FB019C91923008F447C0CA
:108C90008081823008F443C0943051F411961C91C5
:108CA000843099F58181682F70E0611B71093FC0A4
:108CB000843021F0923031F48230B9F181818823FF
:108CC00089F12DC011961C9111978230F1F08181AC
:108CD0001817D9F412962D913C91139782819381A4
:108CE0008217930794F028173907BCF014968D91DA
:108CF0009D910D90BC91A02D248135814681578195
:108D0000281739074A075B0718F4112341F00AC0F6
:108D100082179307A407B50740F4112319F061E007
:108D200070E005C06FEF7FEF02C060E070E0CB0144
:108D30001F910895A0E0B0E0E0EAF6E40C94924AB6
:108D4000EC01A880B980CA80DB80A114B104C10401
:108D5000D10441F484E2A82E89EDB82E8BE5C82E0B
:108D600087E0D82EC601B5012DE133EF41E050E098
:108D70000E94E04A27EA31E440E050E00E94C14A04
:108D80007B018C01C601B5012DE133EF41E050E0DC
:108D90000E94E04ACA01B9012CEE34EF4FEF5FEFB9
:108DA0000E94C14A6E0D7F1D801F911F97FF04C056
:108DB0006150704080409048688379838A839B83A8
:108DC0009B013F77C901CDB7DEB7EAE00C94AE4A0C
:108DD0000E949A4608958CE093E00E949A46089576
:108DE000A0E0B0E080930C0390930D03A0930E03DA
:108DF000B0930F030895FC0188279927E8942191E7
:108E00002032E9F3293010F02E30C8F32B3241F034
:108E10002D3239F4689404C00E948347820F911D5B
:108E2000219120532A30C0F31EF4909581959F4FD5
:108E30000895FB01DC0102C005900D9241505040A5
:108E4000D8F70895FB01DC014150504030F08D917E
:108E50000590801919F40020B9F7881B990B089523
:108E6000FB01DC014150504048F005900D9200207C
:108E7000C9F701C01D9241505040E0F70895FB0131
:108E8000DC0104C08D910190801921F441505040C3
:108E9000C8F7881B990B0895FB01DC0102C0019003
:108EA0000D9241505040D8F708956817790768F43B
:108EB000FB01DC01E40FF51FA40FB51F02C00290F7
:108EC0000E9241505040D8F708950C944C47A0E0C2
:108ED000B0E0EDE6F7E40C94944A7C01EB018A01E2
:108EE000690109C0CE012196F6010995F701819328
:108EF0007F010150104001151105A1F7CDB7DEB774
:108F0000E8E00C94B04A7AE0979F902D879F802DDF
:108F1000910D11240895A0E0B0E0E1E9F7E40C948C
:108F20009A4AFE01359661917191A091A013B0917A
:108F3000A11313968C911397886013968C9380914C
:108F4000A0139091A113AF010E94E647E091A013F6
:108F5000F091A1132381277F23832096E2E00C94D4
:108F6000B64A0F931F93CF93DF938C01E091A01328
:108F7000F091A113838181FF21C0C0E0D0E00DC03A
:108F8000E091A013F091A11320853185BF01F90173
:108F90000995892B11F0CFEFDFEFF80181918F0157
:108FA000882371F7E091A013F091A11320853185FA
:108FB0008AE0BF01F9010995892B11F0CFEFDFEFAE
:108FC000CE01DF91CF911F910F910895ABE0B0E0FA
:108FD000ECEEF7E40C948A4A3C012B015A01FC01A7
:108FE00017821682838181FD03C06FEF7FEFC6C1B8
:108FF0009AE0892E1E010894211C311CF301238163
:10900000F20123FD859123FF81912F01882309F42B
:10901000B2C1853239F423FD859123FF81912F015F
:10902000853229F490E0B3010E94D949E7CF982F07
:10903000FF24EE249924FFE1FF15D0F09B3269F064
:109040009C3228F4903259F0933291F40EC09D3244
:1090500049F0903369F441E024C052E0F52A84E0FD
:10906000F82A28C098E0F92A25C0E0E1FE2A22C0AB
:10907000F7FC29C0892F80538A3070F4F6FE05C0B2
:10908000989C902C1124980E15C0E89CE02C11247B
:10909000E80EF0E2FF2A0EC09E3229F4F6FC6BC106
:1090A00040E4F42A07C09C3619F450E8F52A02C0BF
:1090B000983649F4F20123FD959123FF91912F01F8
:1090C000992309F0B8CF892F8554833018F0805246
:1090D000833038F444E050E0A40EB51E5FE35983BA
:1090E0000FC0933631F0933779F0933509F056C0BD
:1090F00020C0F5018081898342E050E0A40EB51EB6
:10910000610101E010E012C0F501C080D180F6FCE1
:1091100003C06FEF7FEF02C0692D70E042E050E0C6
:10912000A40EB51EC6010E94CE498C015FE7F52250
:1091300014C0F501C080D180F6FC03C06FEF7FEF53
:1091400002C0692D70E042E050E0A40EB51EC601D9
:109150000E94C3498C0150E8F52AF3FE07C01AC0EB
:1091600080E290E0B3010E94D949EA948E2D90E00C
:1091700008171907A8F30EC0F601F7FC8591F7FE52
:1091800081916F0190E0B3010E94D949E110EA9406
:10919000015010400115110579F7EAC0943611F01D
:1091A000993669F5F7FE08C0F501208131814281C9
:1091B000538184E090E00AC0F501808191819C0197
:1091C000442737FD4095542F82E090E0A80EB91E49
:1091D0009FE6F92257FF09C050954095309521959B
:1091E0003F4F4F4F5F4FE0E8FE2ACA01B901A1018E
:1091F0002AE030E00E94054AD82ED21840C09537A8
:1092000029F41F2D1F7E2AE030E01DC01F2D197F7D
:109210009F3661F0903720F4983509F0ACC00FC04C
:10922000903739F0983709F0A6C004C028E030E044
:109230000AC0106114FD146020E130E004C014FD88
:10924000166020E132E017FF08C0F50160817181EE
:109250008281938144E050E008C0F50180819181D2
:10926000BC0180E090E042E050E0A40EB51EA101F8
:109270000E94054AD82ED2188FE7F82EF122F6FE6A
:109280000BC05EEFF522D91438F4F4FE07C0F2FCEF
:1092900005C08FEEF82202C01D2D01C0192DF4FE6D
:1092A0000DC0FE01ED0DF11D8081803319F499EEA2
:1092B000F92208C01F5FF2FE05C003C08F2D86781B
:1092C00009F01F5F0F2DF3FC14C0F0FE0FC01E1538
:1092D00010F09D2C0BC09D2C9E0C911A1E2D06C0CB
:1092E00080E290E0B3010E94D9491F5F1E15C0F3D0
:1092F00004C01E1510F4E11A01C0EE2404FF0FC0D3
:1093000080E390E0B3010E94D94902FF1DC001FD36
:1093100003C088E790E00EC088E590E00BC0802F86
:10932000867891F001FF02C08BE201C080E2F7FC79
:109330008DE290E0B3010E94D94906C080E390E03D
:10934000B3010E94D9499A94D914C0F3DA94F10177
:10935000ED0DF11D808190E0B3010E94D949DD201F
:10936000A9F706C080E290E0B3010E94D949EA94CF
:10937000EE20C1F743CEF30166817781CB012B96B6
:10938000E2E10C94A64AFC01059061507040011086
:10939000D8F7809590958E0F9F1F0895FC0161501E
:1093A000704001900110D8F7809590958E0F9F1F07
:1093B00008950F931F93CF93DF938C01EB018B8163
:1093C00081FF1BC082FF0DC02E813F818C819D815A
:1093D0002817390764F4E881F9810193F983E88358
:1093E00006C0E885F985802F0995892B31F48E8197
:1093F0009F8101969F838E8302C00FEF1FEFC801EC
:10940000DF91CF911F910F910895FA01AA2728307B
:1094100051F1203181F1E8946F936E7F6E5F7F4F41
:109420008F4F9F4FAF4FB1E03ED0B4E03CD0670FBD
:10943000781F891F9A1FA11D680F791F8A1F911D10
:10944000A11D6A0F711D811D911DA11D20D009F460
:1094500068943F912AE0269F11243019305D3193A2
:10946000DEF6CF010895462F4770405D4193B3E08B
:109470000FD0C9F7F6CF462F4F70405D4A3318F032
:10948000495D31FD4052419302D0A9F7EACFB4E0E3
:10949000A6959795879577956795BA95C9F700979B
:1094A0006105710508959B01AC010A2E069457953C
:1094B000479537952795BA95C9F7620F731F841F93
:1094C000951FA01D089597FB092E07260AD077FD4A
:1094D00004D00CD006D000201AF4709561957F4F0F
:1094E0000895F6F7909581959F4F0895AA1BBB1B91
:1094F00051E107C0AA1FBB1FA617B70710F0A61B94
:10950000B70B881F991F5A95A9F780959095BC01B4
:10951000CD0108952F923F924F925F926F927F926A
:109520008F929F92AF92BF92CF92DF92EF92FF9273
:109530000F931F93CF93DF93CDB7DEB7CA1BDB0B1F
:109540000FB6F894DEBF0FBECDBF09942A883988C4
:1095500048885F846E847D848C849B84AA84B984CB
:10956000C884DF80EE80FD800C811B81AA81B981D7
:10957000CE0FD11D0FB6F894DEBF0FBECDBFED01EB
:109580000895629FD001739FF001829FE00DF11D4D
:10959000649FE00DF11D929FF00D839FF00D749F6D
:1095A000F00D659FF00D9927729FB00DE11DF91F19
:1095B000639FB00DE11DF91FBD01CF011124089576
:1095C00097FB092E05260ED057FD04D014D00AD0E3
:1095D000001C38F450954095309521953F4F4F4FE2
:1095E0005F4F0895F6F790958095709561957F4F40
:1095F0008F4F9F4F0895A1E21A2EAA1BBB1BFD019E
:109600000DC0AA1FBB1FEE1FFF1FA217B307E40761
:10961000F50720F0A21BB30BE40BF50B661F771FB9
:10962000881F991F1A9469F7609570958095909599
:0E9630009B01AC01BD01CF010895F894FFCF5E
:10963E00000000000000B2019C0100000143444301
:10964E002070726F636573730000000D01D3060006
:10965E00000000524E4449532070726F636573735D
:10966E000000002301F5070000000001238392781B
:10967E0034200000ADBA01005553422070726F6362
:10968E006573730000004801F6110000000053746A
:10969E006F726167652070726F636573730000008F
:1096AE005E0187140000000016D3200000000000A9
:1096BE00000000000000003830322E31352E3420EC
:1096CE004D41432070726F63657373000000870114
:1096DE00D322000000004576656E742074696D65B6
:1096EE0072000000A60108260000000065746832B2
:1096FE006C6F773A205061636B6574206973206ECE
:10970E006F7420495076362C2064726F7070696EBB
:10971E0067003F3E3D3C3B3A000000000002000067
:10972E000000A536000000006F00000000FE29FEBC
:10973E0016FEC40A00000000000000000001020234
:10974E0003030303040404040404040405050505CB
:10975E0005050505050505050505050506060606A7
:10976E00060606060606060606060606060606068B
:10977E000606060606060606060606060707070777
:10978E00070707070707070707070707070707075B
:10979E00070707070707070707070707070707074B
:1097AE00070707070707070707070707070707073B
:1097BE000707070707070707070707070808080827
:1097CE00080808080808080808080808080808080B
:1097DE0008080808080808080808080808080808FB
:1097EE0008080808080808080808080808080808EB
:1097FE0008080808080808080808080808080808DB
:10980E0008080808080808080808080808080808CA
:10981E0008080808080808080808080808080808BA
:10982E0008080808080808080808080808080808AA
:10983E0008080808080808080808080801000000B9
:020000021000EC
:10FC00000F931F93DB01CA0140E050E0280F391F1A
:10FC10004A1F5B1F81E00801F90140935B0080935C
:10FC20005700E89511241F910F9108950F931F938A
:10FC300083E0F80120935B0080935700E89507B6B6
:10FC400000FCFDCF81E180935700E8951F910F9153
:10FC500008950F931F9385E0F80120935B00809334
:10FC60005700E89507B600FCFDCF81E1809357006F
:08FC7000E8951F910F91089522
:00000001FF
